:1000000016C3000033C3000031C300002FC300003B
:100010002DC300002BC3000029C3000027C300002C
:1000200025C3000023C3000021C300001FC300003C
:100030000C949F3F1BC3000019C3000017C30000AE
:1000400015C3000013C300000C948B3F0FC30000C6
:100050000DC300000BC3000009C3000007C300006C
:1000600005C3000003C3000001C30000FFC200007D
:10007000FDC20000FBC20000F9C20000F7C2000090
:10008000F5C20000F3C20000F1C20000180A1D0A08
:100090002B0A300A350A3A0A3F0A440AD20DD70D14
:1000A000E50DEA0DEF0DF40DF90DFE0DF512F81248
:1000B000FB12FE120113041307130A13501F751FBE
:1000C000891F9C1F9F1FB01FC11FDF1F661F691F55
:1000D000D21FD51FD81F6C1F6F1F721F05251B2530
:1000E0002F2547255D2573259725AD25C3258E270B
:1000F000FB2728299329BB2AF02BDE2CDC2D142F7B
:10010000652FCF2F1A3024308530E030E330E630D1
:10011000E930EC30EF30F230F530A733BD33D33374
:10012000EA33003416342C344234963499349C34F7
:100130009F34A234A534A834AB3403357F35FB3566
:1001400084360D37843700386A38D4384D39BA3997
:10015000313AB73A3A3B00000000000000000404C6
:100160000404000400000A0A0A00000000000A0A51
:100170001F0A1F0A0A00040F140E051E0400181996
:100180000204081303000C12140814120D000C04CE
:100190000800000000000204080808040200080427
:1001A0000202020408000004150E150400000004F9
:1001B000041F04040000000000000C0408000000FC
:1001C000001F0000000000000000000C0C000001F7
:1001D0000204081000000E11131519110E00040C72
:1001E000040404040E000E11010204081F001F0283
:1001F000040201110E0002060A121F0202001F1063
:100200001E0101110E000608101E11110E001F0123
:100210000204080808000E11110E11110E000E1133
:10022000110F01020C000001020408100000000C74
:100230000C000C040800020408100804020000006E
:100240001F001F00000008040201020408000E1134
:100250000102040004000E11010D15150E000E110F
:1002600011111F1111001E11111E11111E000E116E
:10027000101010110E001C12111111121C001F1071
:10028000101E10101F001F10101E101010000E1155
:10029000101711110E001111111F111111000E0470
:1002A000040404040E000702020202120C001112E0
:1002B0001418141211001010101010101F00111B30
:1002C00015151111110011111915131111000E112D
:1002D000111111110E001E11111E101010000E111F
:1002E000111115120D001E11111E141211000F1004
:1002F000100E01011E001F04040404040400111167
:10030000111111110E0011111111110A0400111116
:10031000111115150E0011110A040A111100111105
:10032000110A040404001F01020408101F000E0833
:10033000080808080E00110A1F041F0404000E021A
:10034000020202020E00040A110000000000000078
:10035000000000001F000804000000000000000072
:100360000E010F110F0010101E1111111E000000C0
:100370000E1010110E0001010D1311110F000000DD
:100380000E111F100E000609081C08080800000FB7
:1003900011110F010E001010161911111100040097
:1003A0000C0404040E000200060202120C001010DD
:1003B0001214181412001808080808081C0000007D
:1003C0001A15151111000000161911111100000065
:1003D0000E1111110E0000001E111E101000000061
:1003E0000F110F010100000016191010100000007D
:1003F0000E100E011E0008081C0808090600000067
:10040000111111130D0000001111110A0400000058
:10041000111111150A000000110A040A1100000050
:1004200011110F010E0000001F0204081F003844C4
:1004300044447C4444007C40407844447800784400
:100440004478444478007C404040404040000C14D4
:10045000242424243C447C40407840407C00545474
:100460005438545454003844041804443800444464
:100470004C546444440054444C5464444400444840
:100480005060504844001C24242424246400446CFC
:100490005454444444004444447C44444400384458
:1004A0004444444438007C44444444444400784434
:1004B00044784040400038444040404438007C107C
:1004C0001010101010004444443C044438003854C8
:1004D0005454381010004444281028444400444424
:1004E000444444447E02444444443C040400545480
:1004F000545454547C005454545454547E02602038
:100500002038242438004444446454546400404057
:100510004078444478003844041C0444380048546B
:100520005474545448003C44443C14244400000097
:1005300038043C443C0000007840784478000000D7
:10054000784C784C78000000784040404000000033
:10055000182828287C44000038447C403C000000D7
:1005600054543854540000007804380478000000D3
:10057000444C546444000010444C54644400000053
:1005800044487048440000001C24444444000000D7
:10059000446C545444000000484878484800000027
:1005A0003844444438000000784848484800000077
:1005B0007048704040000000384040403800000063
:1005C0007C1010101000000048483808700000002F
:1005D000385454381000000044281028440000000B
:1005E000484848487C040000484838080800000093
:1005F000545454547C000000545454547E0200005F
:1006000060203C223C0000004242724A720000001E
:1006100040407844780000007008780870000000BE
:100620004C5272524C0000003C443C4444001124A3
:100630001FBECFEFD0E1DEBFCDBF15E0A0E0B1E03F
:10064000E0E2F0E900E00BBF02C007900D92A63E89
:10065000B107D9F726E0A6EEB5E001C01D92A33A96
:10066000B207E1F70E94FD3F0C940E48C9CCE2E6C8
:10067000F0E090819E7F9083908194609083908140
:10068000977F9083A8988BBB8DE08A95F1F7000047
:10069000A89A8081886080830895E2E6F0E09081E6
:1006A000916090839081946090839081977F9083F4
:1006B000A8988BBB8DE08A95F1F70000A89A8081FD
:1006C000886080830895CF93C82F892FE6DF8C2F11
:1006D000CF91E3CFE2E6F0E020812160208320810A
:1006E000246020832081277F2083A8988BBB92BB26
:1006F0008DE08A95F1F70000A89A80818860808358
:100700000895CF93C82F86E3B2DFC13049F030F0AF
:10071000C23041F0C33059F488EE07C088E403C00A
:1007200088E203C088E8B9DF04C0B7DF0BC0CD7F23
:1007300049F48FEE90E09093E9058093E8058FE30C
:1007400091E008C08FE391E09093E9058093E8057C
:100750008FEE90E09093E7058093E605CF910895A2
:10076000CF93C82F8FEF8ABB81BB8093610081E05C
:1007700084BBE2E6F0E080818260808381E077DF05
:100780002FEF89E698E1215080409040E1F700C0CA
:10079000000080EC6CDF85E280DF81EC68DF81E1C6
:1007A0007CDF85EC64DF8BE278DF8BE276DF87EC41
:1007B0005EDF86E872DF8C2FA4DF8AE358DF85E0F6
:1007C0006CDF81EB54DF80E068DF88E166DF86EB79
:1007D0004EDF8AE062DF82E860DF87E25EDF81E190
:1007E00046DF2FEF8DEE92E0215080409040E1F700
:1007F00000C0000089E2CF913ACF0F931F93CF93AF
:10080000DF938C01EB018AE232DFC8015CDFCE01AD
:10081000DF91CF911F910F9156CF0F931F93CF93DD
:10082000DF938C01EB018BE222DFC8014CDFCE01AC
:10083000DF91CF911F910F9146CFCF93DF93EB01C3
:10084000BC01DBDFBE01CE01E8DF8CE2DF91CF919E
:100850000ECFCF93DF93EA01F0DFCE01DF91CF918E
:1008600039CF8F929F92AF92BF92CF92DF92EF9249
:10087000FF920F931F93CF93DF93A8956817790783
:1008800038F4862797276827792786279727A895FA
:100890002417350738F442275327242735274227C2
:1008A0005327A895A091E805B091E905FC01A81788
:1008B000B90708F4FD016B01A617B70708F46D012D
:1008C0008091E6059091E705EA018417950708F401
:1008D000EC0179018217930708F47C01A895960131
:1008E0002F5F3F4F2E1B3F0BD7011196AC1BBD0B4B
:1008F0000E94D6444B015C01B601CF017EDFA89572
:10090000B701CE018ADF8CE2B2DEA895C12CD12CD2
:100910007601C814D904EA04FB0449F0C801DADE00
:10092000A8958FEFC81AD80AE80AF80AF2CFDF9123
:10093000CF911F910F91FF90EF90DF90CF90BF90DC
:10094000AF909F908F9008950F931F93411551057D
:1009500079F02115310561F0FA01AB01615071099F
:10096000260F371FBC01615071096E0F7F1F79DFA1
:100970001F910F9108952F923F924F925F926F9225
:100980007F928F929F92AF92BF92CF92DF92EF921F
:10099000FF920F931F93CF93DF93CDB7DEB7679787
:1009A0000FB6F894DEBF0FBECDBF5C01798B688BAC
:1009B000598748873B872A870F83F12C28E0029FBD
:1009C000C00111241A821982E8E0F0E0FF8BEE8B5F
:1009D00047019C01285F31093B8B2A8BFC01E052C7
:1009E000F340FD8BEC8BC888D98889819A81C80E29
:1009F000D91E8A899B89EE89FF898E1B9F0B9C01DA
:100A00002A5A3E4F3F872E878C899D898E1B9F0BCC
:100A1000FC01EA5AFE4FFD87EC871E821D821C8274
:100A20001B8287E0682E712C412C512C212C312CFB
:100A3000FF81F7FD1EC0EE85FF85849190E0062CB6
:100A400002C0959587950A94E2F780FF08C0088553
:100A500019859701A701B6018D819E8107C00A857E
:100A60001B859701A701B6018B819C818A0D9B1D77
:100A700020C0FF81F03CF0F0EC85FD85849190E092
:100A8000062C02C0959587950A94E2F780FF09C06D
:100A9000088519859701A701B601C501820D931D2F
:100AA00008C00A851B859701A701B601C501840D01
:100AB000951D4ADF280C391C480C591CF1E06F1AAF
:100AC00071082B813C81280D391D3C832B838D813E
:100AD0009E81880D991D9E838D839FEF69167906EF
:100AE00009F0A6CFEE89FF893197FF8BEE8B298124
:100AF0003A812E0D3F1D3A832983EF2B09F073CFE6
:100B000067960FB6F894DEBF0FBECDBFDF91CF91D1
:100B10001F910F91FF90EF90DF90CF90BF90AF901B
:100B20009F908F907F906F905F904F903F902F900D
:100B300008954F925F926F927F928F929F92AF92A1
:100B4000BF92CF92DF92EF92FF920F931F93CF93BA
:100B5000DF93EC016B014A013901102F88E0089FF7
:100B6000500111242701F20101912F010023B1F05E
:100B70002091E8053091E905CE010896281739073C
:100B800020F4CA0CDB1CC1E0D0E0E12E9301A401EB
:100B9000B601CE01F0DECA0DDB1DE5CFDF91CF91AE
:100BA0001F910F91FF90EF90DF90CF90BF90AF908B
:100BB0009F908F907F906F905F904F9008956F926D
:100BC0007F928F929F92AF92BF92CF92DF92EF92DD
:100BD000FF920F93CF93DF9300D000D0CDB7DEB755
:100BE0006C015B014A013901C70119821A821B821B
:100BF0001C824AE0BE016F5F7F4F0E94E544CE0138
:100C000001967C019301A401B501C60192DF0F900A
:100C10000F900F900F90DF91CF910F91FF90EF9079
:100C2000DF90CF90BF90AF909F908F907F906F900C
:100C300008950F931F932091E6053091E705609189
:100C4000E8057091E9058C0140E050E080E090E01B
:100C500008DE1F910F910895EF92FF920F931F935B
:100C6000CF93DF93EB018A017901BC01640F751FFB
:100C7000C4DDBE01CE01D1DD8CE2F9DCC0E0D0E004
:100C8000C017D10721F0C70125DD2196F9CFDF91EB
:100C9000CF911F910F91FF90EF900895EF92FF92E7
:100CA0000F931F93CF93DF93EB018A017901BC016E
:100CB000A4DDBE01600F711FCE01AFDD8CE2D7DC79
:100CC000C0E0D0E0C017D10721F0C70103DD2196B5
:100CD000F9CFDF91CF911F910F91FF90EF90089581
:100CE0002F923F924F925F926F927F928F929F923C
:100CF000AF92BF92CF92DF92EF92FF920F931F932A
:100D0000CF93DF9300D000D000D0CDB7DEB76C0119
:100D10007B015A0139012801261B370B3A832983AD
:100D20008A01081B190B17FF03C0119501951109C2
:100D3000CA14DB0420F022242A94322C03C022247B
:100D40002394312C89819A819E838D8397FF05C0DE
:100D50009195819591099E838D832D813E81319559
:100D6000219531093C832B83E614F70428F08FEF9B
:100D70009FEF9A83898304C021E030E03A8329837E
:100D800048018D819E81881A990AA201B701C60186
:100D900060DDC401880F991F2B813C818217930766
:100DA00064F0CA14DB0499F02D813E81821A930A03
:100DB000C20CD31C0817190744F3E614F70439F0E2
:100DC000800E911E89819A81E80EF91EDECF26964B
:100DD0000FB6F894DEBF0FBECDBFDF91CF911F914C
:100DE0000F91FF90EF90DF90CF90BF90AF909F90CA
:100DF0008F907F906F905F904F903F902F900895CD
:100E0000AF92BF92CF92DF92EF92FF920F931F9318
:100E1000CF93DF937C016B01EA01590198011CDF3C
:100E2000B501615071096C0D7D1D9801AE01C701BE
:100E300013DF9801A501B601C70130DFCE0101978C
:100E40009801A501B6018E0D9F1DDF91CF911F91D5
:100E50000F91FF90EF90DF90CF90BF90AF901ECF9B
:100E60002F923F924F925F926F927F928F929F92BA
:100E7000AF92BF92CF92DF92EF92FF920F931F93A8
:100E8000CF93DF931C012B01690150E0002711274C
:100E9000041B150BC1E0D0E0C41BD50BCC0FDD1F2C
:100EA000E12CF12CA6015701A40CB51CB5013101B0
:100EB000601A710AC301CDDCA601B5014801820C9C
:100EC000931CC401C6DCA6015201AE18BF08B501CF
:100ED000C401BFDCA601B501C301BBDCEC16FD06F5
:100EE000B4F08FEFE81AF80AC701880F991F01962E
:100EF0008C0F9D1F22273327201B310BE216F30690
:100F000039F40C171D074CF0C0E0D0E001C0CE0151
:100F10000C171D0714F0EC01C5CF0F5F1F4F980190
:100F2000220F331F2F5F3F4F820F931F10161106A2
:100F300094F7DF91CF911F910F91FF90EF90DF9089
:100F4000CF90BF90AF909F908F907F906F905F9069
:100F50004F903F902F9008954F925F926F927F92A3
:100F60008F929F92AF92BF92CF92DF92EF92FF92B9
:100F70000F931F93CF93DF93EC015B014A0139017B
:100F800028018601ADDE9701A201B301C401A8DEEC
:100F90009501AE01B701C201A3DEDF91CF911F9190
:100FA0000F91FF90EF90DF90CF90BF90AF909F9008
:100FB0008F907F906F905F904F900895CF93C82F40
:100FC0008A3011F48DE0FADF5D9BFECFCCB980E072
:100FD00090E0CF910895CF92DF92EF92FF920F931E
:100FE0001F93A8950FEF1FEF21E430E04FE550E08D
:100FF00065E070E085E090E003DFA89521E430E053
:101000004FE550E06BE470E085E090E0F9DE2BE422
:1010100030E04FE550E061E970E085E090E0F0DE1F
:10102000A3E3EA2EA5E0FA2E01E02FE130E04FEF36
:101030005FEF60E570E082E190E07BDDBEE2EB2EE9
:10104000B5E0FB2E2FE130E04FEF5FEF6AE570E097
:1010500083E290E06EDD0FEF1FEF21E430E04FE51B
:1010600050E065E070E08CED90E0CADE21E430E015
:101070004FE550E06BE470E08CED90E0C1DE2BE4D6
:1010800030E04FE550E061E970E08CED90E0B8DED3
:1010900013E3E12E15E0F12E01E02FE130E04FEFF8
:1010A0005FEF60E570E08BEE90E043DD88E2E82ED4
:1010B00085E0F82E2FE130E04FEF5FEF6AE570E05A
:1010C0008CEF90E036DD99E5E92E92E0F92E2FE1E4
:1010D00030E04FEF5FEF66EE70E08AE090E029DDF0
:1010E000A89580912B0690912C06019709F04FC08E
:1010F0000FE110E024E430E048E550E064E970E0FE
:1011000088E090E021DC2CE430E04EE650E06CE832
:1011100070E089E690E018DC24E430E048E550E037
:1011200064E970E080EE90E00FDC20EE37E048E20A
:1011300064EB70E080EA90E093DE20EE37E047E277
:1011400064EB70E080EA90E08BDE20EE37E04BE26B
:1011500064EB70E080EA90E083DE20EE37E045E269
:1011600064EB70E080EA90E07BDEE0EECE2EE7E01C
:10117000DE2EF4EBEF2EF12C07EB10E028EC30E044
:1011800044E950E060EA70E084E990E0E5DEA8958B
:1011900080912B0690912C06892B09F051C00FE10C
:1011A00010E024E430E048E550E064E970E088E0D5
:1011B00090E0CADB2CE430E04EE650E06CE870E0F2
:1011C00089E690E0C1DB24E430E048E550E064E9E2
:1011D00070E080EE90E0B8DB20E038EF48E264EBAE
:1011E00070E080EA90E03CDE20E038EF47E264EB1C
:1011F00070E080EA90E034DE20E038EF4BE264EB10
:1012000070E080EA90E02CDE20E038EF45E264EB0D
:1012100070E080EA90E024DE00E018EF23E230E0A6
:1012200045E050E065EA70E086E990E08DDB23E27E
:1012300030E045E050E065EA70E085EA90E084DB6C
:10124000A89580912D0690912E06892B79F4A8956A
:101250007EE1E72E75E0F72E01E02FE130E04FEF61
:101260005FEF63E270E08AE090E063DC80912D063E
:1012700090912E060197E1F4A89557EDE52E55E0E3
:10128000F52E01E02FE130E04FEF5FEF64E170E019
:1012900084E190E04EDC61EDE62E65E0F62E2FE174
:1012A00030E04FEF5FEF68E270E08EE190E041DC0C
:1012B000A89580912D0690912E060297E1F4A895AD
:1012C0003AECE32E35E0F32E01E02FE130E04FEF72
:1012D0005FEF64E170E084E190E02BDC41EDE42E0F
:1012E00045E0F42E2FE130E04FEF5FEF68E270E071
:1012F0008EE190E01EDCA89580912D0690912E063F
:10130000039779F4A89523ECE22E25E0F22E01E074
:101310002FE130E04FEF5FEF63E270E089E190E0B2
:1013200008DCA89580912D0690912E06049779F4FB
:10133000A89594EEE92E94E0F92E01E02FE130E03B
:101340004FEF5FEF63E270E08FE090E0F2DBA89593
:1013500080912D0690912E060597E1F4A8950EED4B
:10136000E02E04E0F02E01E02FE130E04FEF5FEFE0
:1013700064E170E089E190E0DCDB84EDE82E84E05C
:10138000F82E2FE130E04FEF5FEF63E270E08FE087
:1013900090E0CFDBA89580912D0690912E060697C0
:1013A000E1F4A895BEEDEB2EB4E0FB2E01E02FE1B9
:1013B00030E04FEF5FEF64E170E089E190E0B9DB8E
:1013C00012ECE12E14E0F12E2FE130E04FEF5FEF51
:1013D00063E270E08FE190E0ACDBA89580912D0690
:1013E00090912E06079779F4A895A9EAEA2EA4E031
:1013F000FA2E01E02FE130E04FEF5FEF63E270E0A3
:101400008FE090E096DB80912D0690912E06892B3F
:1014100009F048C0A895E0918A068E2F90E08830A8
:10142000910508F03FC0FC01EA5BFF4F0C94CD44EE
:10143000F4EAEF2EF4E0FF2E04C0EFE9EE2EE4E034
:10144000FE2E02E02FE130E04FEF5FEF6EE170E043
:101450008BEE90E026C075E9E72E74E0F72E18C0F9
:101460006BE8E62E64E0F62E13C051E8E52E54E05A
:10147000F52E0EC047E7E42E44E0F42E09C03DE609
:10148000E32E34E0F32E04C023E6E22E24E0F22E15
:1014900001E02FE130E04FEF5FEF6EE170E086EEAC
:1014A00090E047DB80912D0690912E06019701F583
:1014B000A89580913606813069F038F08230C1F409
:1014C00001E8E02E04E0F02E09C095E9E92E94E051
:1014D000F92E04C08BE8E82E84E0F82E01E02FE11D
:1014E00030E04FEF5FEF6EE170E086EE90E021DBE1
:1014F00080912D0690912E06029701F5A895809176
:101500003D06813069F038F08230C1F4A1E8EA2E5E
:10151000A4E0FA2E09C015E9E12E14E0F12E04C072
:10152000BBE8EB2EB4E0FB2E01E02FE130E04FEF03
:101530005FEF6EE170E086EE90E0FBDA80912D06C1
:1015400090912E06039779F4A895FFEEEF2EF4E024
:10155000FF2E01E02FE130E04FEF5FEF6EE170E032
:101560008EEE90E0E6DA80912D0690912E0604979B
:1015700001F5A89580919506813069F038F08230A8
:10158000C1F461E8E62E64E0F62E09C0E5E9EE2E2E
:10159000E4E0FE2E04C07BE8E72E74E0F72E01E0C5
:1015A0002FE130E04FEF5FEF6EE170E086EE90E00C
:1015B000C0DA80912D0690912E06059701F5A89529
:1015C00080918906813069F038F08230C1F431E8C9
:1015D000E32E34E0F32E09C055E9E52E54E0F52E54
:1015E00004C04BE8E42E44E0F42E01E02FE130E0AB
:1015F0004FEF5FEF6EE170E086EE90E09ADA809157
:101600002D0690912E06069701F5A89580918606E5
:10161000813069F038F08230C1F481E8E82E84E04E
:10162000F82E09C025E9E22E24E0F22E04C09BE842
:10163000E92E94E0F92E01E02FE130E04FEF5FEF6B
:101640006EE170E086EE90E074DA80912D06909164
:101650002E06079709F4A8951F910F91FF90EF9020
:10166000DF90CF900895CF92DF92EF92FF920F9389
:101670001F93A89500EE17E021E430E048EC50E01D
:101680006AEA70E085E090E05FD90FEF1FEF21E498
:1016900030E048EC50E063E270E085E090E0B0DBE1
:1016A00087E7E82E82E0F82E01E02FE130E040EEFF
:1016B00057E06CE370E088E290E03BDA0FEF1FEF59
:1016C00020E530E040E550E065E070E08BEE90E032
:1016D00097DB90EEC92E97E0D92E24E1E22EF12C73
:1016E00003E111E026E430E041E351E066E470E01C
:1016F00085EF90E031DC37E1E32EF12C24E430E09B
:101700004FE251E064E470E087EF90E025DC0FEFFA
:101710001FEF20E530E040E550E064E670E08BEE3E
:1017200090E06EDB45EAE42EF12C03E111E023E7C3
:1017300030E041E351E063E770E085EF90E00CDCDE
:1017400053EAE52EF12C25E730E04FE251E065E762
:1017500070E087EF90E000DC66E4E62E65E0F62EB0
:1017600002E020EE37E040E050E068EC70E08DE20F
:1017700090E0DFD91F910F91FF90EF90DF90CF9015
:101780000895CF92DF92EF92FF920F931F93A89547
:1017900000EE17E021E430E048EC50E06AEA70E047
:1017A00085E090E0D1D80FEF1FEF21E430E048EC66
:1017B00050E063E270E085E090E022DB83EBE82E0E
:1017C00084E0F82E01E02FE130E040EE57E06CE3DA
:1017D00070E088E290E0ADD90FEF1FEF20E530E038
:1017E00040E550E065E070E08BEE90E009DB90EEC4
:1017F000C92E97E0D92E24E1E22EF12C03E111E06D
:1018000026E430E041E351E066E470E085EF90E0EB
:10181000A3DB37E1E32EF12C24E430E04FE251E08A
:1018200064E470E087EF90E097DB0FEF1FEF20E5B7
:1018300030E040E550E064E670E08BEE90E0E0DA06
:1018400045EAE42EF12C03E111E023E730E041E327
:1018500051E063E770E085EF90E07EDB53EAE52E30
:10186000F12C25E730E04FE251E065E770E087EFCB
:1018700090E072DB6FEDE62E65E0F62E02E020EEE2
:1018800037E040E050E068EC70E08DE290E051D944
:101890001F910F91FF90EF90DF90CF900895CF921E
:1018A000DF92EF92FF920F931F93A89500EE17E03F
:1018B00021E430E048EC50E06AEA70E085E090E036
:1018C00043D80FEF1FEF21E430E048EC50E063E233
:1018D00070E085E090E094DA82E5E82E84E0F82E6E
:1018E00001E02FE130E040EE57E06CE370E088E289
:1018F00090E01FD90FEF1FEF20E530E040E550E00A
:1019000065E070E08BEE90E07BDA90EEC92E97E018
:10191000D92E24E1E22EF12C03E111E026E430E09F
:1019200041E351E066E470E085EF90E015DB37E1DC
:10193000E32EF12C24E430E04FE251E064E470E067
:1019400087EF90E009DB0FEF1FEF20E530E040E587
:1019500050E064E670E08BEE90E052DA45EAE42E67
:10196000F12C03E111E023E730E041E351E063E7CC
:1019700070E085EF90E0F0DA53EAE52EF12C25E7F0
:1019800030E04FE251E065E770E087EF90E0E4DAA5
:1019900067E5E62E65E0F62E02E020EE37E040E057
:1019A00050E068EC70E08DE290E0C3D81F910F9199
:1019B000FF90EF90DF90CF900895CF93DF9300D00A
:1019C00000D0CDB7DEB7809163001C821B821A82E3
:1019D0001982BE016F5F7F4FCE0103960E94304394
:1019E0008B819C818431954068F489819A81843A05
:1019F000964040F489819A818D32914018F082E0BE
:101A0000809353068B819C818937954090F08B8120
:101A10009C81843C994068F489819A81843A9640FB
:101A200040F489819A818D32914018F083E080934F
:101A300053068B819C8189329A4068F089819A8112
:101A400084379E4040F489819A81813D974018F007
:101A500081E0809353068B819C81863F994060F49E
:101A60008B819C818134964038F089819A81813DB7
:101A7000974010F010925306809153060F900F90EC
:101A80000F900F90DF91CF910895CF92DF92EF9258
:101A9000FF920F931F93A89500EE17E021E430E02A
:101AA00048EC50E06AEA70E085E090E00E94A4040F
:101AB0000FEF1FEF21E430E048EC50E063E270E00C
:101AC00085E090E09DD920E530E040E550E065E01C
:101AD00070E08BEE90E094D9F0EECF2EF7E0DF2EA1
:101AE000A4E1EA2EF12C03E111E026E430E041E329
:101AF00051E066E470E085EF90E02EDAB7E1EB2E7E
:101B0000F12C24E430E04FE251E064E470E087EF30
:101B100090E022DA0FEF1FEF20E530E040E550E0E3
:101B200064E670E08BEE90E06BD915EAE12EF12CC3
:101B300003E111E023E730E041E351E063E770E0C7
:101B400085EF90E009DA83EAE82EF12C25E730E012
:101B50004FE251E065E770E087EF90E0FDD99FED3F
:101B6000E92E95E0F92E02E020EE37E040E050E06B
:101B700068EC70E08CE390E00E94990580912D065E
:101B800090912E06892B09F048C0E0918A068E2F8D
:101B900090E08830910508F040C0FC01E25BFF4F07
:101BA0000C94CD44E4EAEE2EE4E0FE2E04C07FE97E
:101BB000E72E74E0F72E02E02FE130E04FEF5FEF09
:101BC00065E070E086E490E026C065E9E62E64E01A
:101BD000F62E18C05BE8E52E54E0F52E13C041E860
:101BE000E42E44E0F42E0EC037E7E32E34E0F32E6B
:101BF00009C02DE6E22E24E0F22E04C093E6E92E81
:101C000094E0F92E02E02FE130E04FEF5FEF65E066
:101C100070E08EE190E00E94990580912D069091F0
:101C20002E06019701F580913606813069F038F073
:101C30008230C9F411E8E12E14E0F12E09C085E9E3
:101C4000E82E84E0F82E04C00BE8E02E04E0F02E2D
:101C500002E02FE130E04FEF5FEF65E070E08EE1F2
:101C600090E00E94990580912D0690912E06029792
:101C700001F580913D06813069F038F08230C9F479
:101C8000F1E8EF2EF4E0FF2E09C0B5E9EB2EB4E049
:101C9000FB2E04C0ABE8EA2EA4E0FA2E02E02FE10E
:101CA00030E04FEF5FEF65E070E08EE190E00E9482
:101CB000990580912D0690912E06049701F580914B
:101CC0009506813069F038F08230C9F461E8E62E7B
:101CD00064E0F62E09C0E5E9EE2EE4E0FE2E04C035
:101CE0007BE8E72E74E0F72E02E02FE130E04FEFC3
:101CF0005FEF65E070E08EE190E00E9499058091D1
:101D00002D0690912E06059701F580918906813068
:101D100069F038F08230C9F431E8E32E34E0F32E74
:101D200009C055E9E52E54E0F52E04C04BE8E42E39
:101D300044E0F42E02E02FE130E04FEF5FEF65E08A
:101D400070E08EE190E00E94990580912D069091BF
:101D50002E06069701F580918606813069F038F0ED
:101D60008230C9F481E8E82E84E0F82E09C025E924
:101D7000E22E24E0F22E04C09BE8E92E94E0F92E36
:101D800002E02FE130E04FEF5FEF65E070E08EE1C1
:101D900090E00E9499051F910F91FF90EF90DF90C6
:101DA000CF900895EF92FF920F931F938091240696
:101DB000909125060A97A8F48091FB0581110CC02B
:101DC0000FE110E02CE330E044E650E06BE470E01B
:101DD0008EE690E00E94A40481E08093FB051092BF
:101DE0002F0680912406909125060A978A35910541
:101DF000A8F480912F0681110CC00FE110E02CE3B4
:101E000030E044E650E06BE470E08EE690E00E9443
:101E1000A40481E080932F061092FB058091240694
:101E20009091250684369105A0F080912F0681308F
:101E300061F40FE110E02CE330E044E650E06BE4A5
:101E400070E08EE690E00E94A40410922F0610929B
:101E5000FB0580912B0690912C06019779F4E09078
:101E60002406F090250603E02FE130E04FEF5FEF0E
:101E700064E670E082E890E00E94DF0580912B0626
:101E800090912C06892B79F4E0902406F090250699
:101E900003E02FE130E040E058EF64E670E082E8D4
:101EA00090E00E94DF051F910F91FF90EF90089541
:101EB000EF92FF920F931F938091570690915806CF
:101EC0000A97A8F480912306811111C00FE110E058
:101ED00027E330E048E550E06BE970E088E090E00F
:101EE0000E94A40481E080932306109287068091CB
:101EF00057069091580684369105D8F480912406AF
:101F0000909125060A97A8F080918706811111C04B
:101F10000FE110E027E330E048E550E06BE970E0C6
:101F200088E090E00E94A40481E0809387061092EC
:101F30002306809157069091580684369105A0F0AB
:101F400080918706813061F40FE110E027E330E0F3
:101F500048E550E06BE970E088E090E00E94A4045E
:101F60001092870610922306E0905706F0905806CC
:101F700003E02FE130E04FEF5FEF64EB70E08FE0C4
:101F800090E00E94DF051F910F91FF90EF90089560
:101F9000EF92FF920F931F93809144069091450614
:101FA0000A97A8F480912A0681110CC00FE110E075
:101FB00024E230E04AE550E064E670E088E090E03A
:101FC0000E94A40481E080932A0610924106809129
:101FD0004406909145060A978A359105A8F48091A8
:101FE000410681110CC00FE110E024E230E04AE527
:101FF00050E064E670E088E090E00E94A40481E094
:102000008093410610922A068091440690914506DD
:1020100084369105A1F480914106813061F40FE18D
:1020200010E024E230E04AE550E064E670E088E049
:1020300090E00E94A40410922A061092410680911A
:102040004406909145068436910530F084E690E090
:102050009093450680934406E0904406F090450630
:1020600003E02FE130E04FEF5FEF6EE670E084E1D8
:1020700090E00E94DF0580919606909197060A975E
:10208000A8F480919006811111C00FE110E024E2C4
:1020900030E04AE550E064E670E08FED90E00E94A9
:1020A000A40481E0809390061092590680919606D0
:1020B000909197060A978A359105A8F48091590660
:1020C000811111C00FE110E024E230E04AE550E058
:1020D00064E670E08FED90E00E94A40481E08093BC
:1020E0005906109290068091960690919706843634
:1020F000910529F4109290061092590603C0843677
:10210000910530F084E690E09093970680939606D0
:10211000E0909606F090970603E02FE130E04FEF55
:102120005FEF6EE670E089EE90E00E94DF051F91A0
:102130000F91FF90EF900895CF93DF9300D000D0E0
:10214000CDB7DEB7809163001C821B821A82198290
:10215000BE016F5F7F4FCE0103960E9430438B819B
:102160009C81853C9940A0F0A89589819A81843C06
:10217000994070F4A89589819A818D3D954040F0F1
:10218000A89581E090E090932C0680932B06A8956B
:102190000F900F900F900F90DF91CF910895CF93F4
:1021A000DF9300D000D0CDB7DEB7A8958091630053
:1021B0001C821B821A821982BE016F5F7F4FCE0183
:1021C00003960E9430438B819C81853C9940A8F006
:1021D00089819A81843C994080F489819A818D3DDE
:1021E000954058F010922C0610922B068FE19EE439
:1021F0000197F1F700C00000A8950F900F900F9085
:102200000F90DF91CF9108957F928F929F92AF921E
:10221000BF92CF92DF92EF92FF920F931F93CF93D3
:10222000DF93EC016B015A014901702EA895809152
:10223000FE059091FF050A97A8F480918B06811105
:1022400011C00FE110E02EE130E044E650E06550AF
:102250007109CE0144970E94A40481E080938B060B
:1022600010924C068091FE059091FF050A978A35E1
:102270009105C0F480914C06811114C00FE110E06B
:102280002EE130E044E650E0B60165507109CE0120
:1022900044970E94A40481E080934C0610928B0620
:1022A000109226068091FE059091FF0584369105D7
:1022B000C0F080912606811114C00FE110E02EE1DC
:1022C00030E044E650E0B60165507109CE01449714
:1022D0000E94A40481E08093260610924C0610927E
:1022E0008B06E090FE05F090FF05072D9401A501F7
:1022F000B601CE010E94DF05A895DF91CF911F9115
:102300000F91FF90EF90DF90CF90BF90AF909F9094
:102310008F907F900895CF92DF92EF92FF920F936C
:102320001F938FE190E00E941906A89500EE17E038
:1023300021E430E048EC50E06AEA70E085E090E0AB
:102340000E94A4040FEF1FEF21E430E048EC50E0BE
:1023500063E270E085E090E00E94000789E4E82EE7
:1023600082E0F82E01E02FE130E040EE57E06CE330
:1023700070E088E290E00E9499050FEF1FEF20E5E2
:1023800030E040E550E065E070E08BEE90E00E94C8
:10239000000790EEC92E97E0D92E24E1E22EF12C11
:1023A00003E111E026E430E041E351E066E470E04F
:1023B00085EF90E00E94AC0737E1E32EF12C24E496
:1023C00030E04FE251E064E470E087EF90E00E947B
:1023D000AC070FEF1FEF20E530E040E550E064E68A
:1023E00070E08BEE90E00E94000745EAE42EF12CAD
:1023F00003E111E023E730E041E351E063E770E0FF
:1024000085EF90E00E94AC0753EAE52EF12C25E71A
:1024100030E04FE251E065E770E087EF90E00E9426
:10242000AC0766E4E62E65E0F62E02E020EE37E02B
:1024300040E050E068EC70E08DE290E00E94990589
:102440008FE19EE40197F1F700C000001F910F910A
:10245000FF90EF90DF90CF900895A8958091490666
:10246000813071F4A49A80E185BBA8952FEF82E5B5
:1024700097E0215080409040E1F700C0000015BA7D
:10248000A8950895A89580914906813021F5A49AD0
:1024900080E185BB2FEF32E597E02150304090403E
:1024A000E1F700C00000A89515BA2FEF32E597E0DC
:1024B000215030409040E1F700C00000A89585BB56
:1024C0002FEF32E587E0215030408040E1F700C037
:1024D0000000A89515BA0895A89580914906813005
:1024E00009F048C0A49A80E185BBA8952FEF32E59A
:1024F00097E0215030409040E1F700C00000A895DF
:1025000015BAA8952FEF32E597E021503040904062
:10251000E1F700C00000A89585BBA8952FEF32E534
:1025200097E0215030409040E1F700C00000A895AE
:1025300015BAA8952FEF32E597E021503040904032
:10254000E1F700C00000A89585BB2FEF32E587E0DA
:10255000215030408040E1F700C00000A89515BA36
:102560009FEF22E537E0915020403040E1F700C076
:102570000000A8950895A8951092460610923A0674
:102580001092FA0510925C061092370610922906F6
:102590001092480610924006109256061092EB05D3
:1025A00083EB92E00E94E84780934906A89584EB6C
:1025B00092E00E94F04790933C0680933B06A895DA
:1025C00080912D0690912E06892B51F5A895E091CA
:1025D0008A068E2F90E08830910510F5FC01EA5AAA
:1025E000FF4F4EE150E00C94CD4464E972E014C01A
:1025F00066E772E011C068E572E00EC06AE372E05F
:102600000BC06CE172E008C06EEF71E005C060EED7
:1026100071E002C062EC71E084E096E00E94D8476D
:10262000A89580912D0690912E060197D1F4A8953A
:1026300080913606813069F038F0823091F44EE1B5
:1026400050E068E671E009C04EE150E064EA71E0F4
:1026500004C04EE150E066E871E084E096E00E943C
:10266000D847A89580912D0690912E060297D1F417
:10267000A89580913D06813069F038F0823091F460
:102680004EE150E06EE071E009C04EE150E06AE4D6
:1026900071E004C04EE150E06CE271E084E096E04D
:1026A0000E94D847A89580912D0690912E060497F8
:1026B000C9F480919506813069F038F0823091F448
:1026C0004EE150E064EB70E009C04EE150E060EF95
:1026D00070E004C04EE150E062ED70E084E096E00E
:1026E0000E94D847A89580912D0690912E060597B7
:1026F000C9F480918906813069F038F0823091F414
:102700004EE150E06AE570E009C04EE150E066E954
:1027100070E004C04EE150E068E770E084E096E0CD
:102720000E94D847A89580912D0690912E06069775
:10273000C9F480918606813069F038F0823091F4D6
:102740004EE150E060E070E009C04EE150E06CE323
:1027500070E004C04EE150E06EE170E084E096E08D
:102760000E94D847A89587EC90E00197F1F700C048
:10277000000080910406909105069093F9058093DE
:10278000F805809106069091070690934B0680937A
:102790004A068091080690910906909393068093CB
:1027A000920680910A0690910B06909335068093CD
:1027B000340680910C0680935F0680910E069091FE
:1027C0000F06909333068093320680911006809313
:1027D00043068091120680934206809114068093EE
:1027E000F4058091160690911706909383068093C6
:1027F0008206809118069091190690935E06809348
:102800005D0680912D0690912E06079741F48091E8
:102810001A0690911B0690932E0680932D068091A8
:102820001C0690911D0690938106809380068091EE
:102830001E0690911F0690930306809302068091D6
:102840002006909121069093280680932706A8954C
:1028500008951092970610929606BC9A809196065B
:10286000880F81BF1092450610924406139A8091FA
:102870004406880F809386002FDE8DE490E09093CD
:102880008D0680938C0681E090E090932C068093D7
:102890002B060895CF934091FE055091FF0520919E
:1028A000340630913506429FC001439F900D529FE0
:1028B000900D11246AE070E00E94B94470935B06A9
:1028C00060935A068091440690914506853691059D
:1028D00030F084E690E09093450680934406809122
:1028E000420690E0209144063091450682179307F6
:1028F00020F49093450680934406209146062111CA
:1029000014C02091570630915806283C310538F400
:1029100024E630E0309345062093440606C0283C68
:10292000310519F021E0209346062091460640919A
:102930004A0650914B062130E1F520914406309132
:1029400045062436310530F024E630E03093450664
:10295000209344066417750760F5E0915706F091DF
:1029600058062091440630914506E617F707C0F453
:102970002F5F3F4F8217930728F03093450620932F
:10298000440604C090934506809344062091440673
:10299000309145062536310560F024E630E005C06B
:1029A0002115310531F0215031093093450620932E
:1029B00044064617570708F04AC020915706309141
:1029C000580624173507D0F46091440670914506E7
:1029D0006F5F7F4F6536710510F064E670E07093AD
:1029E000450660934406609144067091450686173B
:1029F000970720F4909345068093440642175307A7
:102A000030F58091440690914506009729F0019792
:102A10009093450680934406241B350B2B303105DB
:102A2000B0F080914406909145060A9720F41092E8
:102A300045061092440680914406909145068A30DE
:102A4000910528F00A979093450680934406C0911B
:102A50005F06C130D9F480913A06811117C02091E8
:102A6000240630912506809132069091330628176E
:102A7000390760F0F2DC8091570690915806C297B2
:102A800090934B0680934A06C0933A06C091F40592
:102A9000C13009F58091FA0581111DC0809124068D
:102AA000909125062091820630918306821B930B1C
:102AB000059788F420914A0630914B0680915D0677
:102AC00090915E06820F931F90934B0680934A0667
:102AD000C4DCC093FA05CF91089580915C06811102
:102AE0001CC08091240690912506209132063091D9
:102AF0003306821B930B029780F482E390E090935D
:102B000097068093960681E080935C068093290661
:102B100080915F06811101C0A0DC8091EA052091BF
:102B2000320630913306811119C060918E06709182
:102B30008F064091920650919306649FC001659F55
:102B4000900D749F900D11246AE070E00E94B944CA
:102B5000620F731F7093F7056093F6054091F805B7
:102B60005091F9058091F6059091F705481759079E
:102B700038F45093F7054093F60581E08093EA0519
:102B80008091430690E060919606709197068617B3
:102B9000970720F4909397068093960680912406D9
:102BA000909125062817390720F048175907A0F1FA
:102BB00076C0209156062111F8CF84179507A8F703
:102BC0006091F6057091F705209196063091970671
:102BD0008617970788F42F5F3F4F2536310528F475
:102BE0003093970620939606E0CF24E630E03093AA
:102BF000970620939606A6C02115310531F0215085
:102C000031093093970620939606209196063091CD
:102C10009706232B51F296C0209196063091970685
:102C20002115310531F02150310930939706209359
:102C30009606841B950B0697B0F0809196069091AE
:102C400097060A9720F410929706109296068091A4
:102C50009606909197068A30910528F00A979093EE
:102C60009706809396068091EB05811106C00ADCD9
:102C700081E0809340068093EB052091000630911F
:102C8000010680913B0690913C068217930738F429
:102C9000E0DD81E090E090932C0680932B068091FC
:102CA0003706811158C0409180065091810680916D
:102CB0003206909133068417950708F04CC0E091D6
:102CC0002406F09125064E175F0729F481E08093D2
:102CD000560680934806809156068130E1F5609152
:102CE000FC057091FD0520910206309103066217E4
:102CF0007307A8F48091960690919706E417F5075C
:102D000038F401968536910530F084E690E003C0F2
:102D1000009729F0019790939706809396062617BF
:102D20003707C8F41092560680918E0690918F0650
:102D3000821B930B90938F0680938E0681E0809385
:102D4000370608954817590708F0A9CF209196062D
:102D50003091970668CF089580915C0681111BC061
:102D600020912406309125068091320690913306F9
:102D70008217930780F482E390E090939706809304
:102D8000960681E080935C068093290680915F0619
:102D9000811101C062DBE0913206F091330640916F
:102DA0008E0650918F062091920630919306429F95
:102DB000C001439F900D529F900D11246AE070E076
:102DC0000E94B9446E0F7F1F7093F7056093F6055C
:102DD00020919606309197064091F8055091F9059B
:102DE0004617570720F45093F7054093F605809156
:102DF000430690E08217930720F490939706809300
:102E000096062091240630912506E217F30700F577
:102E10008091560681111CC024173507C8F46091B3
:102E2000F6057091F7058091960690919706261702
:102E3000370738F401968536910530F084E690E046
:102E400003C0009729F00197909397068093960608
:102E500042175307E0F580919606909197060197E7
:102E60009093970680939606241B350B26303105E8
:102E700090F00A9720F4109297061092960680918F
:102E80009606909197068A30910528F00A979093BC
:102E90009706809396068091EB05811106C0F2DAC1
:102EA00081E0809340068093EB05209100063091ED
:102EB000010680913B0690913C068217930738F4F7
:102EC000C8DC81E090E090932C0680932B068091E3
:102ED000370681114EC04091800650918106809145
:102EE0003206909133068417950708F042C0E091AE
:102EF0002406F09125064E175F0729F481E08093A0
:102F000056068093480680915606813091F560916F
:102F1000FC057091FD0520910206309103066217B1
:102F20007307A8F48091960690919706E417F50729
:102F300038F401968536910530F084E690E003C0C0
:102F4000009729F00197909397068093960626178D
:102F5000370778F41092560680918E0690918F066E
:102F6000821B930B90938F0680938E0681E0809353
:102F700037060895CF93C0915F06C130D1F4809198
:102F80003A06811116C020912406309125068091C1
:102F90003206909133062817390759F48091570665
:102FA0009091580690934B0680934A0656DAC09348
:102FB0003A064091FE055091FF052091340630916C
:102FC0003506429FC001439F900D529F900D1124E2
:102FD0006AE070E00E94B94470935B0660935A0601
:102FE00080914406909145068536910530F084E63F
:102FF00090E090934506809344068091420690E0CD
:1030000020914406309145068217930720F490934F
:1030100045068093440620914606211114C0209154
:103020005706309158062639310538F424E630E049
:10303000309345062093440606C02639310519F021
:1030400021E0209346062091460640914A06509181
:103050004B06213079F56417750760F5E091570646
:10306000F09158062091440630914506E617F7077F
:10307000C0F42F5F3F4F8217930728F03093450627
:103080002093440604C09093450680934406209103
:103090004406309145062536310560F024E630E0DF
:1030A00005C02115310531F0215031093093450615
:1030B000209344064617570708F088C020915F0602
:1030C000211133C020915706309158062417350737
:1030D000D0F460914406709145066F5F7F4F65366E
:1030E000710510F064E670E0709345066093440645
:1030F00060914406709145068617970720F49093D7
:103100004506809344064217530708F05FC080913C
:10311000440690914506009729F001979093450643
:1031200080934406241B350B38C0213009F04EC073
:103130002091240630912506609132067091330665
:1031400026173707D0F440914406509145064F5F4B
:103150005F4F4536510510F044E650E05093450668
:1031600040934406409144065091450684179507C4
:1031700020F490934506809344066217730730F558
:103180008091440690914506009729F0019790930D
:10319000450680934406261B370B2B303105B0F0D3
:1031A00080914406909145060A9720F410924506B6
:1031B0001092440680914406909145068A3091050C
:1031C00028F00A979093450680934406CF9108957E
:1031D0004091FE055091FF0520913406309135064F
:1031E000429FC001439F900D529F900D11246AE0B1
:1031F00070E00E94B94470935B0660935A06809118
:103200004406909145068536910530F084E690E0BD
:1032100090934506809344068091420690E0209169
:103220004406309145068217930720F49093450693
:1032300080934406209146064091570650915806C7
:10324000211110C04639510538F424E630E030939E
:1032500045062093440606C04639510519F021E081
:103260002093460620914606E0914A06F0914B06CF
:10327000213059F56E177F0740F5209144063091B3
:10328000450646175707C0F42F5F3F4F8217930735
:1032900028F0309345062093440604C090934506D9
:1032A0008093440620914406309145062536310529
:1032B00060F024E630E005C02115310531F02150E1
:1032C00031093093450620934406E617F70708F0C6
:1032D00046C04E175F07D0F4209144063091450652
:1032E0002F5F3F4F2536310510F024E630E0309354
:1032F00045062093440620914406309145068217E6
:10330000930720F49093450680934406E417F5074D
:1033100030F58091440690914506009729F0019779
:103320009093450680934406CA018E1B9F0B0B9712
:10333000B0F080914406909145060A9720F41092CF
:1033400045061092440680914406909145068A30C5
:10335000910528F00A979093450680934406809142
:10336000430690E0209196063091970682179307C6
:1033700020F49093970680939606E417F50770F46F
:10338000809196069091970601968536910510F0EA
:1033900084E690E090939706809396060895409176
:1033A000FE055091FF052091340630913506429F6D
:1033B000C001439F900D529F900D11246AE070E070
:1033C0000E94B94470935B0660935A06809144064C
:1033D000909145068536910530F084E690E0909313
:1033E0004506809344068091420690E02091440671
:1033F000309145068217930720F4909345068093F9
:10340000440620914606211114C0209157063091A0
:1034100058062639310538F424E630E03093450665
:103420002093440606C02639310519F021E0209387
:1034300046062091460640914A0650914B0621309F
:1034400079F56417750760F5E0915706F091580615
:103450002091440630914506E617F707C0F42F5F28
:103460003F4F8217930728F0309345062093440678
:1034700004C0909345068093440620914406309101
:1034800045062536310560F024E630E005C02115FB
:10349000310531F02150310930934506209344061F
:1034A0004617570708F04AC0209157063091580632
:1034B00024173507D0F460914406709145066F5F7C
:1034C0007F4F6536710510F064E670E07093450635
:1034D00060934406609144067091450686179707ED
:1034E00020F490934506809344064217530730F525
:1034F0008091440690914506009729F0019790939A
:10350000450680934406241B350B2B303105B0F063
:1035100080914406909145060A9720F41092450642
:103520001092440680914406909145068A30910598
:1035300028F00A9790934506809344060895BC9A14
:1035400080919606880F81BF139A80914406880F58
:103550008093860080912D0690912E06892B11F480
:1035600099D9BBDA80912D0690912E06019729F406
:103570001092450610924406EFDB80912D06909143
:103580002E06029729F41092970610929606F2DC06
:1035900080912D0690912E06049709F419DE8091F2
:1035A0002D0690912E06059709F412DE80912D06C6
:1035B00090912E06069709F4F2CE089563EC70E020
:1035C00084E992E00E940B4862EC71E086E992E0A7
:1035D0000E940B4866E170E088E992E00E940B4887
:1035E00066E170E08AE992E00E940B4861E070E0D9
:1035F0008CE992E00E940B48A8956EE670E08EE997
:1036000092E00E940B4864E670E080EA92E00E943B
:103610000B4864E670E082EA92E00E940B4860E0AA
:1036200070E084EA92E00E940B48A89560E070E0A8
:1036300086EA92E00E940B4860E070E088EA92E03F
:103640000E940B4860E070E08AEA92E00E940B481A
:1036500060E070E08CEA92E00E940B4860E070E06D
:103660008EEA92E00E940B4860E070E080EB92E00E
:103670000E940B48A89566EE70E086E792E00E94F3
:103680000B4862EC71E088E792E00E940B4866E12B
:1036900070E08AE792E00E940B4866E170E08CE7F8
:1036A00092E00E940B4861E070E08EE792E00E9499
:1036B0000B48A89563E770E080E892E00E940B4811
:1036C00064E670E082E892E00E940B4864E670E0F5
:1036D00084E892E00E940B4860E070E086E892E0A7
:1036E0000E940B4860E070E088E892E00E940B487E
:1036F00060E070E08AE892E00E940B48A89560E0E4
:1037000070E08CE892E00E940B4860E070E08EE888
:1037100092E00E940B4860E070E080E992E00E9435
:103720000B4860E070E082E992E00E940B48A895A7
:1037300066EE70E088E592E00E940B4862EC71E072
:103740008AE592E00E940B4866E170E08CE592E029
:103750000E940B4866E170E08EE592E00E940B4803
:1037600061E070E080E692E00E940B48A89563E774
:1037700070E082E692E00E940B4864E670E084E626
:1037800092E00E940B4864E670E086E692E00E94B8
:103790000B4860E070E088E692E00E940B4860E031
:1037A00070E08AE692E00E940B4860E070E08CE6F0
:1037B00092E00E940B48A89560E070E08EE692E0EF
:1037C0000E940B4860E070E080E792E00E940B48A6
:1037D00060E070E082E792E00E940B4860E070E0F9
:1037E00084E792E00E940B48A89566E970E08AE3BE
:1037F00092E00E940B4868EC70E08CE392E00E943B
:103800000B4866E170E08EE392E00E940B4866E1AF
:1038100070E080E492E00E940B4861E070E082E496
:1038200092E00E940B48A89563E770E084E492E080
:103830000E940B4864E670E086E492E00E940B4828
:1038400064E670E088E492E00E940B4860E070E07B
:103850008AE492E00E940B4860E070E08CE492E021
:103860000E940B4860E070E08EE492E00E940B48FA
:10387000A89560E070E080E592E00E940B4860E06F
:1038800070E082E592E00E940B4860E070E084E521
:1038900092E00E940B4860E070E086E592E00E94B2
:1038A0000B48A8956EEB70E08CE192E00E940B480B
:1038B00068EC70E08EE192E00E940B4866E170E0F7
:1038C00080E292E00E940B4866E170E082E292E0C2
:1038D0000E940B4861E070E084E292E00E940B4895
:1038E000A89564E670E086E292E00E940B4864E6E8
:1038F00070E088E292E00E940B4864E670E08AE2A1
:1039000092E00E940B4860E070E08CE292E00E943E
:103910000B4860E070E08EE292E00E940B4860E0AD
:1039200070E080E392E00E940B48A89560E070E0B0
:1039300082E392E00E940B4860E070E084E392E052
:103940000E940B4860E070E086E392E00E940B4822
:1039500060E070E088E392E00E940B48A89566EE74
:1039600070E08EEF91E00E940B4862EC71E080E025
:1039700092E00E940B4866E170E082E092E00E94D3
:103980000B4866E170E084E092E00E940B4861E041
:1039900070E086E092E00E940B48A89563E770E033
:1039A00088E092E00E940B4864E670E08AE092E0D2
:1039B0000E940B4864E670E08CE092E00E940B48A5
:1039C00060E070E08EE092E00E940B4860E070E002
:1039D00080E192E00E940B4860E070E082E192E0BA
:1039E0000E940B48A89560E070E084E192E00E949C
:1039F0000B4860E070E086E192E00E940B4860E0D6
:103A000070E088E192E00E940B4860E070E08AE19B
:103A100092E00E940B48A89566EE70E080EE91E07F
:103A20000E940B4862EC71E082EE91E00E940B482C
:103A300066E170E084EE91E00E940B4866E170E080
:103A400086EE91E00E940B4861E070E088EE91E024
:103A50000E940B48A89563E770E08AEE91E00E940F
:103A60000B4864E670E08CEE91E00E940B4864E63F
:103A700070E08EEE91E00E940B4860E070E080EF15
:103A800091E00E940B4860E070E082EF91E00E94BC
:103A90000B4860E070E084EF91E00E940B48A8952D
:103AA00060E070E086EF91E00E940B4860E070E01B
:103AB00088EF91E00E940B4860E070E08AEF91E0AF
:103AC0000E940B4860E070E08CEF91E00E940B4890
:103AD000A89563EC70E084EA91E00E940B4866E1EF
:103AE00070E088EA91E00E940B4861E070E08CEAA7
:103AF00091E00E940B486FE070E08EEA91E00E9436
:103B00000B48A89564E670E080EB91E00E940B48BA
:103B100061E070E08AEB91E00E940B4863EC70E09A
:103B20008CEB91E00E940B486AE070E08EEB91E034
:103B30000E940B48A89562EC71E08CE491E00E9431
:103B40000B4866E170E080E591E00E940B4861E07F
:103B500070E082E591E00E940B486EE670E084E53B
:103B600091E00E940B48A89564E670E088E591E03A
:103B70000E940B4862E070E080E691E00E940B48F2
:103B800062EC71E082EF90E00E940B4866E170E029
:103B900084EF90E00E940B4862E170E086EF90E0D5
:103BA0000E940B48A89564E670E08CEF90E00E94BC
:103BB0000B4864E670E08EEF90E00E940B4864E0F2
:103BC00070E086E091E00E940B486CE271E08CE0CE
:103BD00091E00E940B48A89562EC71E088E990E0C2
:103BE0000E940B4866E170E08AE990E00E940B4871
:103BF00066E170E08CE990E00E940B4861E070E0C3
:103C00008EE990E00E940B48A8956EE670E080EA8D
:103C100090E00E940B4864E670E082EA90E00E9427
:103C20000B4864E670E084EA90E00E940B4865E08F
:103C300070E08CEA90E00E940B48A89562EC71E07D
:103C40008EE390E00E940B4866E170E082E490E031
:103C50000E940B4861E070E084E490E00E940B4811
:103C60006EE670E086E490E00E940B48A89564E65A
:103C700070E08AE490E00E940B4866E070E082E524
:103C800090E00E940B4863EC70E084E992E00E94AF
:103C90000B48A89508956FE070E088EB92E00E94D1
:103CA0000B486FE070E086EB92E00E940B486FE0FB
:103CB00070E084EB92E00E940B4861E083EB92E0BD
:103CC0000E94FE4761E082EB92E00C94FE478FB9C0
:103CD000779BFECF8FB10895CF93A39AAB9AAB9801
:103CE00080E0F5DFC82F80E0F2DFAB9A6C2F70E048
:103CF000762F6627682B687F7F7723E07695679518
:103D00002A95E1F780E090E00E94C84320E030E08F
:103D100040E85EE30E942E440E949C437093250677
:103D200060932406CB01CF910895CF93A79AAF9AC1
:103D3000AF9880E0CCDFC82F80E0C9DFAF9A6C2F4E
:103D400070E0762F6627682B687F7F7723E0769573
:103D500067952A95E1F780E090E00E94C84320E053
:103D600030E040E85EE30E942E440E949C43709342
:103D7000580660935706CB01CF91089580E091E0FB
:103D80009093A00680939F06809125068F93809143
:103D900024068F938EE091E09F938F930E940845B5
:103DA0008DE08A95F1F700008091FF058F93809157
:103DB000FE058F9388E191E09F938F930E940845C1
:103DC0009DE09A95F1F70000809145068F938091D0
:103DD00044068F9382E291E09F938F930E9408455F
:103DE0008DE08A95F1F70000809197068F9380917E
:103DF00096068F938DE291E09F938F930E940845E2
:103E00009DE09A95F1F7000087E391E09F938F93EF
:103E10000E9408458DE08A95F1F7000080915806D0
:103E20008F93809157068F938FE391E09F938F93A9
:103E30000E940845A8958DB79EB746960FB6F89490
:103E40009EBF0FBE8DBF80912B0690912C06892BB3
:103E500041F488E491E09F938F930E9408450F906E
:103E60000F90A89580912B0690912C06019741F414
:103E70008FE491E09F938F930E9408450F900F90DD
:103E80009DE09A95F1F70000E0912D06F0912E0645
:103E9000E830F10508F09CC0E25AFF4F0C94CD4485
:103EA00086E591E09F938F930E940845A8950F9017
:103EB0000F90E0918A068E2F90E08830910508F0EF
:103EC00087C0FC01EA59FF4F0C94CD4485E691E090
:103ED00071C085E791E06EC08DEA91E06BC08CEB1C
:103EE00091E068C08BEC91E065C08AED91E09F9312
:103EF0008F930E940845A8950F900F9080913606E9
:103F0000813009F452C008F44DC0823009F450C029
:103F100008958AEE91E09F938F930E940845A8959B
:103F20000F900F9080913D06813009F43EC0D0F192
:103F3000823009F43DC008958BEF91E042C089E0E2
:103F400092E09F938F930E940845A8950F900F9041
:103F500080919506813049F128F1823049F1089528
:103F60008AE192E09F938F930E940845A8950F9055
:103F70000F90809189068130C1F0A0F08230C1F0AD
:103F800008958DE292E09F938F930E940845A89533
:103F90000F900F9080918606813039F018F08230B2
:103FA00039F0089580E891E005C08FE891E002C003
:103FB0008EE991E09F938F930E94084507C08FE39D
:103FC00092E09F938F930E940845A8950F900F90C1
:103FD0000895CF92DF92EF92FF920F931F93CF93AA
:103FE000DF9300D000D0CDB7DEB780912B06909143
:103FF0002C06019709F045C180913E0690913F063D
:10400000892BD9F40FE110E024E230E04AE550E0DA
:1040100064E670E088E090E00E94A40424E230E0CE
:104020004AE550E064E670E08FED90E00E94A40461
:10403000A895A49AAC980E94EB07CC24C394D12CE9
:1040400080912B0690912C06019709F01AC1A89532
:1040500095DE80918C0690918D068A35910549F404
:104060002FEF8DE399E4215080409040E1F700C0AC
:104070000000A89503E02FE130E04FEF5FEF69E12A
:1040800070E085E890E00E94041180916300A8959B
:104090001C821B821A821982BE016F5F7F4FCE0184
:1040A00003960E9430438B819C818431954088F433
:1040B00089819A81883D9E4060F489819A81853CFE
:1040C000994038F0D0923F06C0923E0610924E06BC
:1040D00026D48B819C818431954008F03FC0898132
:1040E0009A818C3D9540D0F589819A81853F914098
:1040F000A8F1D0923F06C0923E06109260068091D1
:104100002D0690912E06892B11F40E942F33809159
:104110002D0690912E06019711F40E94CB3B8091C1
:104120002D0690912E06029711F40E94D23C8091A8
:104130002D0690912E06049711F40E94D93D80918E
:104140002D0690912E06059709F471D580912D06C4
:1041500090912E06069711F40E9427328091F30564
:10416000813019F58B819C81853C9940F0F08981E3
:104170009A818C3D9540C8F489819A81853F914010
:10418000A0F0D0923F06C0923E060E948B1180E0C4
:104190000E94F2410E945C4210923F0610923E063D
:1041A0008FE190E00E94190614DF96DD0E94D20E86
:1041B000A8958FEF91EE24E0815090402040E1F7E8
:1041C00000C00000B2DDA8950E94580FE0904406A0
:1041D000F090450603E02FE130E04FEF5FEF6EE631
:1041E00070E08CE190E00E94DF05E0909606F09090
:1041F00097062FE130E04FEF5FEF6EE670E080EF63
:1042000090E00E94DF058091F305813011F40E9457
:10421000E4420E94CF1080912B0690912C06892BAE
:1042200009F00ECFA8950E94BB12A8950E942D12EE
:104230000E94EB070FE110E024E230E04AE550E095
:1042400064E670E088E090E00E94A40424E230E09C
:104250004AE550E064E670E08FED90E00E94A4042F
:104260008091F305813021F40E94ED410E940043CA
:104270001092FF051092FE0510923F0610923E0626
:10428000DFCE0F900F900F900F90DF91CF911F9185
:104290000F91FF90EF90DF90CF900895EF92FF92F3
:1042A0000F931F93CF9380914D06813009F04BC13E
:1042B0008FE190E00E9419060E94C10B85E0809377
:1042C0005306C5E080914D06813009F03CC10E9443
:1042D000DD0C809153068230D9F480917F068F5F88
:1042E00080937F060FE110E02CE330E046EE50E0D3
:1042F00069E670E081E090E00E94A40422E330E0EF
:1043000043EC50E068E270E088E090E00E94A40492
:10431000809153068330D9F480917F068150809339
:104320007F060FE110E02CE330E046EE50E069E656
:1043300070E081E090E00E94A40422E330E043ECCE
:1043400050E068E270E088E090E00E94A404809170
:104350007F06853010F010927F0680917F068230B4
:1043600081F1B8F48823D9F0813009F0C1C076E931
:10437000E72E75E0F72E01E02FE130E04FEF5FEF21
:104380006CE370E088E090E00E94990586EB92E093
:1043900029C08330B1F1843009F471C0A9C0EFEABB
:1043A000EE2EE5E0FE2E01E02FE130E04FEF5FEF73
:1043B0006CE370E08FE090E00E94990588EB92E05A
:1043C00011C06AE8E62E65E0F62E01E02FE130E04C
:1043D0004FEF5FEF6CE370E082E390E00E9499059D
:1043E00084EB92E00E94F0477C0103E02FE130E093
:1043F0004FEF5FEF62E870E080E590E00E94DF053C
:1044000077C042E7E42E45E0F42E01E02FE130E0F2
:104410004FEF5FEF6CE370E088E290E00E94990557
:1044200050E8E52E55E0F52E02E02FE130E04FEFA9
:104430005FEF62E870E088E290E00E949905809169
:104440005306811119C0BAD826DC3CE3E32E35E0CF
:10445000F32E2FE130E04FEF5FEF62E870E088E28B
:1044600090E00E9499052FEF89E698E12150804065
:104470009040E1F700C00000C093530639C021E628
:10448000E22E25E0F22E01E02FE130E04FEF5FEF6A
:104490006CE370E08EE190E00E94990583EB92E07E
:1044A0000E94E847813079F493E5E92E95E0F92EF2
:1044B00003E02FE130E04FEF5FEF62E870E080E56E
:1044C00090E00E94990583EB92E00E94E8478111F9
:1044D0000FC08EE4E82E85E0F82E03E02FE130E0F7
:1044E0004FEF5FEF62E870E080E590E00E94990591
:1044F00080915306813089F410924D0610923F0648
:1045000010923E068FE190E00E94190681E090E053
:1045100090932C0680932B065CDD809153068111CD
:1045200006C081E080934D061092910612D0C09390
:1045300053062FE785EB91E0215080409040E1F752
:1045400000C00000BFCECF911F910F91FF90EF9060
:104550000895BF92CF92DF92EF92FF920F931F9335
:10456000CF93DF93809191068111CFC185E0809335
:104570005306C9E1D0E025E0C22ED12C35E0B32EA0
:10458000809191068111C1C180917F06813009F42B
:104590006FC038F0823009F4DDC0843009F441C1C5
:1045A000A4C188EB92E00E94F0477C0103E02FE178
:1045B00030E040E058EF62E870E080E590E00E9473
:1045C000DF0588EB92E00E94F047909352068093BB
:1045D00051060E94DD0C809153068230A9F480912F
:1045E000510690915206019690935206809351067F
:1045F0000FE110E02CE330E046EE50E069E670E0B9
:1046000081E090E00E94A404809153068330A9F4D5
:104610008091510690915206019790935206809393
:1046200051060FE110E02CE330E046EE50E069E681
:1046300070E081E090E00E94A40480915106909186
:1046400052064A9720F0D0935206C09351068091AB
:104650005106909152060A9720F4D0935206C093C7
:104660005106609151067091520688EB92E066C047
:1046700086EB92E00E94F0477C0103E02FE130E0FE
:1046800040E058EF62E870E080E590E00E94DF05CE
:1046900086EB92E00E94F0479093310680933006BB
:1046A0000E94DD0C809153068230A9F4809130067F
:1046B00090913106019690933106809330060FE178
:1046C00010E02CE330E046EE50E069E670E081E077
:1046D00090E00E94A404809153068330A9F4809155
:1046E0003006909131060197909331068093300601
:1046F0000FE110E02CE330E046EE50E069E670E0B8
:1047000081E090E00E94A4048091300690913106EF
:104710004A9720F0D0933106C0933006809130063E
:10472000909131060A9720F4D0933106C093300659
:10473000609130067091310686EB92E00E940B4842
:104740002FE788E391E0215080409040E1F700C0DE
:104750000000CBC084EB92E00E94F0477C0103E0B4
:104760002FE130E040E058EF62E870E080E590E053
:104770000E94DF0584EB92E00E94F0479093500680
:1047800080934F060E94DD0C809153068230A9F47D
:1047900080914F0690915006019690935006809319
:1047A0004F060FE110E02CE330E046EE50E069E602
:1047B00070E081E090E00E94A40480915306833071
:1047C000A9F480914F06909150060197909350065E
:1047D00080934F060FE110E02CE330E046EE50E00E
:1047E00069E670E081E090E00E94A40480914F06A9
:1047F000909150064F9720F0D0925006C0924F06ED
:1048000080914F0690915006059720F4D092500663
:10481000C0924F0660914F067091500684EB92E073
:104820008DCF83EB92E00E94E8478093F5050E94CC
:10483000DD0C80915306823089F48091F5058F5FFD
:104840008093F5050FE110E02CE330E046EE50E0F8
:1048500069E670E081E090E00E94A4048091530634
:10486000833089F48091F50581508093F5050FE13F
:1048700010E02CE330E046EE50E069E670E081E0C5
:1048800090E00E94A4048091F505823010F010920F
:10489000F5058091F505813079F493E5E92E95E0F1
:1048A000F92E03E02FE130E040E058EF62E870E0DD
:1048B00080E590E00E9499058091F50581110FC077
:1048C0008EE4E82E85E0F82E03E02FE130E040E0B2
:1048D00058EF62E870E080E590E00E9499056091F1
:1048E000F50583EB92E00E94FE47809153068130EC
:1048F00049F48093910680934D068FE190E00E94E9
:104900001906CCDCB09253063BCEDF91CF911F91BC
:104910000F91FF90EF90DF90CF90BF9008954F924E
:104920005F926F927F928F929F92AF92BF92CF923F
:10493000DF92EF92FF920F931F93CF93DF938091BB
:104940004E06811163C18FE190E00E9419060E941A
:10495000330B85E08093530610924D061092470664
:1049600055245394C7E0D0E0A6E0CA2ED12CB5E080
:10497000AB2EB12C14E0812E912C03E0602E712C13
:1049800085E0482E80914E06811140C10E94DD0CC9
:1049900080915306823089F4809147068F5F80931F
:1049A00047060FE110E02CE330E046EE50E069E608
:1049B00070E081E090E00E94A4048091530683306F
:1049C00089F4809147068150809347060FE110E0FB
:1049D0002CE330E046EE50E069E670E081E090E0E4
:1049E0000E94A40480914706893010F01092470677
:1049F000E09147068E2F90E08930910508F0D4C0F1
:104A0000FC01E259FF4F0C94CD44FEE1EF2EF5E09E
:104A1000FF2E02E02FE130E04FEF5FEF62E870E041
:104A200088E090E00E94990510924D0610922E06A3
:104A300010922D06B9C0E0E1EE2EE5E0FE2E02E078
:104A40002FE130E04FEF5FEF68E770E088E090E043
:104A50000E94990510924D0681E090E013C072E02B
:104A6000E72E75E0F72E02E02FE130E04FEF5FEF29
:104A700068E770E088E090E00E94990510924D068A
:104A800082E090E090932E0680932D068DC066EF15
:104A9000E62E64E0F62E02E02FE130E04FEF5FEF0C
:104AA00068E770E088E090E00E94990510924D065A
:104AB00070922E0660922D0677C054EEE52E54E0DB
:104AC000F52E02E02FE130E04FEF5FEF68E770E096
:104AD00088E090E00E94990510924D0690922E0673
:104AE00080922D0661C03EEDE32E34E0F32E02E00D
:104AF0002FE130E04FEF5FEF6EE670E088E290E08C
:104B00000E94990544EDE42E44E0F42E2FE130E0BC
:104B10004FEF5FEF67E870E08FE090E00E9499054B
:104B200010924D06B0922E06A0922D063DC027ECA5
:104B3000E22E24E0F22E02E02FE130E04FEF5FEFB3
:104B400068E770E088E090E00E94990510924D06B9
:104B5000D0922E06C0922D0627C099EAE92E94E045
:104B6000F92E02E02FE130E04FEF5FEF68E770E0F1
:104B700088E090E00E94990510924D06D0932E0691
:104B8000C0932D0611C083EBE82E84E0F82E02E0DE
:104B90002FE130E04FEF5FEF68E770E082E090E0F8
:104BA0000E94990550924D0680915306813011F56F
:104BB00080914D06813059F410922E0610922D06E8
:104BC00010924E068FE190E00E94190667DB50922A
:104BD0004E0610923F0610923E0680912D0690914F
:104BE0002E0690931B0680931A068FE190E00E9498
:104BF0001906EFD9409253062FEF80E792E021503B
:104C000080409040E1F700C00000BCCEDF91CF9122
:104C10001F910F91FF90EF90DF90CF90BF90AF90DA
:104C20009F908F907F906F905F904F900895EF923C
:104C3000FF920F931F93CF93DF93A8958091600607
:104C40008111F4C08FE190E00E9419060E944F0C80
:104C50008091890690E0909339068093380685E02C
:104C600080935306C1E0D5E0809160068111DEC0DB
:104C7000A8950E94DD0C809153068230A9F48091A2
:104C8000380690913906019690933906809338063C
:104C90000FE110E02CE330E046EE50E069E670E012
:104CA00081E090E00E94A404809153068330A9F42F
:104CB0008091380690913906019790933906809338
:104CC00038060FE110E02CE330E046EE50E069E6F4
:104CD00070E081E090E00E94A404809138069091F9
:104CE0003906039720F01092390610923806809109
:104CF0003806909139068130910589F1D0F00297FC
:104D000009F046C081E8E82E84E0F82E02E02FE1A9
:104D100030E04FEF5FEF6DE770E088E290E00E94D7
:104D2000990582E0809389064EE150E06AE570E0E3
:104D30002BC025E9E22E24E0F22E02E02FE130E044
:104D40004FEF5FEF6DE770E088E290E00E94990519
:104D5000109289064EE150E066E970E015C09BE8CC
:104D6000E92E94E0F92E02E02FE130E04FEF5FEF03
:104D70006DE770E088E290E00E949905C093890693
:104D80004EE150E068E770E084E096E00E94D8478A
:104D90008091530681110FC0A895C09360061092B0
:104DA0003F0610923E06C0934E068FE190E00E94AF
:104DB0001906A8950ED980915306813059F5A8950A
:104DC0008093600610923F0610923E0680934E0636
:104DD0008FE190E00E941906A895109298068091A4
:104DE0008906813069F038F0823091F44EE150E06C
:104DF0006AE570E009C04EE150E066E970E004C089
:104E00004EE150E068E770E084E096E00E94D84709
:104E1000A89513D0D09353062FEF80E792E021504E
:104E200080409040E1F700C000001ECFDF91CF919D
:104E30001F910F91FF90EF900895EF92FF920F93C3
:104E40001F93CF938091980681110C9421328FE1AA
:104E500090E00E9419060E94450D85E0809353065C
:104E6000C5E08091980681110C9421320E94DD0CDE
:104E7000809153068230D9F4809184068F5F8093AD
:104E800084060FE110E02CE330E046EE50E069E6E6
:104E900070E081E090E00E94A40422E330E043EC63
:104EA00050E068E270E088E090E00E94A404809105
:104EB00053068330D9F48091840681508093840610
:104EC0000FE110E02CE330E046EE50E069E670E0E0
:104ED00081E090E00E94A40422E330E043EC50E043
:104EE00068E270E088E090E00E94A404809184066B
:104EF0008E3010F010928406E09184068E2F90E0A0
:104F00008E30910510F00C94C430FC01E958FF4F2D
:104F100080912D0690912E060C94CD44892BB9F5E5
:104F20008091040690910506893E934020F01092EE
:104F30000506109204067BE3E72E74E0F72E01E0ED
:104F40002FE130E04FEF5FEF62E370E08FE090E041
:104F50000E949905E4E3EE2EE4E0FE2E2FE130E01E
:104F60004FEF5FEF66E470E08CE390E00E949905FC
:104F7000E0900406F090050603E02FE130E04FEFEB
:104F80005FEF62E870E080E590E00E94DF058091CD
:104F90002D0690912E06019709F0F1C78091040625
:104FA00090910506893E934020F0109205061092DC
:104FB00004065BE3E52E54E0F52E01E02FE130E03E
:104FC0004FEF5FEF62E370E08FE090E00E949905A1
:104FD00064E3E62E64E0F62E2FE130E04FEF5FEF62
:104FE00066E470E08CE390E00E949905E09004068E
:104FF000F0900506B9C7892BB9F580910606909106
:105000000706893E934020F010920706109206068C
:105010003CE1E32E34E0F32E01E02FE130E04FEFEE
:105020005FEF62E370E08FE090E00E9499054EE050
:10503000E42E44E0F42E2FE130E04FEF5FEF66E422
:1050400070E08CE390E00E949905E0900606F090F5
:10505000070603E02FE130E04FEF5FEF62E870E01A
:1050600080E590E00E94DF0580912D0690912E064C
:105070008130910531F4809184068F5F809384069E
:1050800039C00297B9F58091060690910706893ECE
:10509000934020F010920706109206069CE1E92E3C
:1050A00094E0F92E01E02FE130E04FEF5FEF62E393
:1050B00070E08FE090E00E9499052EE0E22E24E05F
:1050C000F22E2FE130E04FEF5FEF66E470E08CE30B
:1050D00090E00E949905E0900606F090070603E034
:1050E0002FE130E04FEF5FEF62E870E080E590E0A5
:1050F0000E94DF0580912D0690912E060497B9F548
:105100008091060690910706893E934020F0109208
:105110000706109206060CE1E02E04E0F02E01E0F6
:105120002FE130E04FEF5FEF62E370E08FE090E05F
:105130000E9499058EE0E82E84E0F82E2FE130E001
:105140004FEF5FEF66E470E08CE390E00E9499051A
:10515000E0900606F090070603E02FE130E04FEF05
:105160005FEF62E870E080E590E00E94DF058091EB
:105170002D0690912E060597B9F58091060690911F
:105180000706893E934020F010920706109206060B
:10519000BCE1EB2EB4E0FB2E01E02FE130E04FEF5D
:1051A0005FEF62E370E08FE090E00E9499051EE0FF
:1051B000E12E14E0F12E2FE130E04FEF5FEF66E4D7
:1051C00070E08CE390E00E949905E0900606F09074
:1051D000070603E02FE130E04FEF5FEF62E870E099
:1051E00080E590E00E94DF0580912D0690912E06CB
:1051F000069709F0C9C78091060690910706893E77
:10520000934020F01092070610920606FCE1EF2E64
:10521000F4E0FF2E01E02FE130E04FEF5FEF62E3BB
:1052200070E08FE090E00E949905AEE0EA2EA4E0E5
:10523000FA2E2FE130E04FEF5FEF66E470E08CE391
:1052400090E00E949905E0900606F0900706E0C500
:10525000892BB1F580910806909109064F9720F0AF
:10526000109209061092080676EFE72E73E0F72EEB
:1052700001E02FE130E04FEF5FEF62E370E08FE09D
:1052800090E00E949905EEEDEE2EE3E0FE2E2FE178
:1052900030E04FEF5FEF66E470E08FE090E00E9457
:1052A0009905E0900806F090090603E02FE130E050
:1052B0004FEF5FEF62E870E080E590E00E94DF056D
:1052C00080912D0690912E06019709F058C6809185
:1052D0000806909109064F9720F010920906109247
:1052E000080656EFE52E53E0F52E01E02FE130E001
:1052F0004FEF5FEF62E370E08FE090E00E9499056E
:105300006EEDE62E63E0F62E2FE130E04FEF5FEF1B
:1053100066E470E08FE090E00E949905E090080656
:10532000F090090621C6892BB1F580910A0690916B
:105330000B064F9720F010920B0610920A0636ECDF
:10534000E32E33E0F32E01E02FE130E04FEF5FEF8B
:1053500062E370E08FE090E00E9499054EEAE42E4F
:1053600043E0F42E2FE130E04FEF5FEF66E470E0B2
:105370008FE090E00E949905E0900A06F0900B06FD
:1053800003E02FE130E04FEF5FEF62E870E080E58F
:1053900090E00E94DF0580912D0690912E068130CD
:1053A000910531F4809184068F5F8093840638C024
:1053B0000297B1F580910A0690910B064F9720F065
:1053C00010920B0610920A0696ECE92E93E0F92E45
:1053D00001E02FE130E04FEF5FEF62E370E08FE03C
:1053E00090E00E9499052EEAE22E23E0F22E2FE1B2
:1053F00030E04FEF5FEF66E470E08FE090E00E94F6
:105400009905E0900A06F0900B0603E02FE130E0EA
:105410004FEF5FEF62E870E080E590E00E94DF050B
:1054200080912D0690912E060497B1F580910A0681
:1054300090910B064F9720F010920B0610920A06DF
:1054400006ECE02E03E0F02E01E02FE130E04FEF1C
:105450005FEF62E370E08FE090E00E9499058EEAD2
:10546000E82E83E0F82E2FE130E04FEF5FEF66E4A7
:1054700070E08FE090E00E949905E0900A06F090BD
:105480000B0603E02FE130E04FEF5FEF62E870E0E2
:1054900080E590E00E94DF0580912D0690912E0618
:1054A0000597B1F580910A0690910B064F9720F071
:1054B00010920B0610920A06B6ECEB2EB3E0FB2E10
:1054C00001E02FE130E04FEF5FEF62E370E08FE04B
:1054D00090E00E9499051EEAE12E13E0F12E2FE1E3
:1054E00030E04FEF5FEF66E470E08FE090E00E9405
:1054F0009905E0900A06F0900B0603E02FE130E0FA
:105500004FEF5FEF62E870E080E590E00E94DF051A
:1055100080912D0690912E06069709F035C6809150
:105520000A0690910B064F9720F010920B061092EE
:105530000A06F6ECEF2EF3E0FF2E01E02FE130E05B
:105540004FEF5FEF62E370E08FE090E00E9499051B
:10555000AEEAEA2EA3E0FA2E2FE130E04FEF5FEF44
:1055600066E470E08FE090E00E949905E0900A0602
:10557000F0900B064DC4892B09F045C080910C06B4
:1055800090910D06039730F081E090E090930D0626
:1055900080930C06E6E9EE2EE3E0FE2E01E02FE11B
:1055A00030E04FEF5FEF6CE370E08FE090E00E943F
:1055B000990580910C0690910D06019779F473E599
:1055C000E72E75E0F72E03E02FE130E04FEF5FEFBD
:1055D00062E870E080E590E00E94990580910C06F9
:1055E00090910D06892B79F46EE4E62E65E0F62E97
:1055F00003E02FE130E04FEF5FEF62E870E080E51D
:1056000090E00E94990580912D0690912E068130A0
:10561000910509F044C020910C0630910D0623300D
:10562000310520F090930D0680930C0656E9E52E87
:1056300053E0F52E01E02FE130E04FEF5FEF6CE338
:1056400070E08FE090E00E94990580910C069091A7
:105650000D06019779F443E5E42E45E0F42E03E0CE
:105660002FE130E04FEF5FEF62E870E080E590E01F
:105670000E94990580910C0690910D06892B79F472
:105680003EE4E32E35E0F32E03E02FE130E04FEF70
:105690005FEF62E870E080E590E00E9499058091FC
:1056A0002D0690912E06029709F045C080910C06B8
:1056B00090910D06039730F081E090E090930D06F5
:1056C00080930C0626E9E22E23E0F22E01E02FE182
:1056D00030E04FEF5FEF6CE370E08FE090E00E940E
:1056E000990580910C0690910D06019779F493E548
:1056F000E92E95E0F92E03E02FE130E04FEF5FEF68
:1057000062E870E080E590E00E94990580910C06C7
:1057100090910D06892B79F48EE4E82E85E0F82E21
:1057200003E02FE130E04FEF5FEF62E870E080E5EB
:1057300090E00E94990580912D0690912E069C0183
:10574000245031092230310508F4D9C4069709F0F4
:105750001BC580910C0690910D06039730F081E0F7
:1057600090E090930D0680930C0606E9E02E03E08E
:10577000F02E01E02FE130E04FEF5FEF6CE370E0DF
:105780008FE090E00E94990580910C0690910D06A3
:10579000019779F413E5E12E15E0F12E03E02FE1F6
:1057A00030E04FEF5FEF62E870E080E590E00E944C
:1057B000990580910C0690910D06892B09F0E4C49F
:1057C000BEE4EB2EB5E0FB2E03E02FE130E04FEF1F
:1057D0005FEF62E870E080E590E00E949905D4C434
:1057E000892BB9F580910E0690910F068F35914067
:1057F00020F010920F0610920E06FEE7EF2EF3E057
:10580000FF2E01E02FE130E04FEF5FEF62E370E049
:105810008FE090E00E949905A6E6EA2EA3E0FA2E1A
:105820002FE130E04FEF5FEF66E470E08FE090E053
:105830000E949905E0900E06F0900F0603E02FE11C
:1058400030E04FEF5FEF62E870E080E590E00E94AB
:10585000DF0580912D0690912E060197B9F5809174
:105860000E0690910F068F35914020F010920F0692
:1058700010920E067EE7E72E73E0F72E01E02FE18F
:1058800030E04FEF5FEF62E370E08FE090E00E9466
:105890009905E6E6EE2EE3E0FE2E2FE130E04FEF35
:1058A0005FEF66E470E08FE090E00E949905E09081
:1058B0000E06F0900F0603E02FE130E04FEF5FEFB0
:1058C00062E870E080E590E00E94DF0580912D069F
:1058D00090912E060297B9F580910E0690910F06D1
:1058E0008F35914020F010920F0610920E065EE761
:1058F000E52E53E0F52E01E02FE130E04FEF5FEFB2
:1059000062E370E08FE090E00E94990566E6E62E83
:1059100063E0F62E2FE130E04FEF5FEF66E470E0DA
:105920008FE090E00E949905E0900E06F0900F063F
:1059300003E02FE130E04FEF5FEF62E870E080E5D9
:1059400090E00E94DF0580912D0690912E069C012B
:10595000245031092230310508F4D1C3069709F0EB
:1059600013C480910E0690910F068F35914020F060
:1059700010920F0610920E063EE7E32E33E0F32E50
:1059800001E02FE130E04FEF5FEF62E370E08FE086
:1059900090E00E94990546E6E42E43E0F42E2FE1C4
:1059A00030E04FEF5FEF66E470E08FE090E00E9440
:1059B0009905E0900E06F0900F062AC2892BB9F5E2
:1059C00080911006909111068636910520F0109274
:1059D0001106109210069EE4E92E93E0F92E01E0E4
:1059E0002FE130E04FEF5FEF62E370E08FE090E097
:1059F0000E94990526E3E22E23E0F22E2FE130E00B
:105A00004FEF5FEF66E470E08FE090E00E94990551
:105A1000E0901006F090110603E02FE130E04FEF28
:105A20005FEF62E870E080E590E00E94DF05809122
:105A30002D0690912E060197B9F580911006909150
:105A400011068636910520F010921106109210066C
:105A50000EE4E02E03E0F02E01E02FE130E04FEF06
:105A60005FEF62E370E08FE090E00E94990586E3CB
:105A7000E82E83E0F82E2FE130E04FEF5FEF66E491
:105A800070E08FE090E00E949905E0901006F090A1
:105A9000110603E02FE130E04FEF5FEF62E870E0C6
:105AA00080E590E00E94DF0580912D0690912E0602
:105AB0008230910531F4809184068F5F8093840653
:105AC00039C00497B9F58091100690911106863679
:105AD000910520F01092110610921006BEE4EB2EF4
:105AE000B3E0FB2E01E02FE130E04FEF5FEF62E328
:105AF00070E08FE090E00E94990516E3E12E13E03C
:105B0000F12E2FE130E04FEF5FEF66E470E08FE0C1
:105B100090E00E949905E0901006F090110603E0D5
:105B20002FE130E04FEF5FEF62E870E080E590E05A
:105B30000E94DF0580912D0690912E060597B9F5FC
:105B400080911006909111068636910520F01092F2
:105B5000110610921006FEE4EF2EF3E0FF2E01E096
:105B60002FE130E04FEF5FEF62E370E08FE090E015
:105B70000E949905A6E3EA2EA3E0FA2E2FE130E079
:105B80004FEF5FEF66E470E08FE090E00E949905D0
:105B9000E0901006F090110603E02FE130E04FEFA7
:105BA0005FEF62E870E080E590E00E94DF058091A1
:105BB0002D0690912E06A0C2892BB9F58091120670
:105BC000909113068636910520F0109213061092DC
:105BD00012067EE1E72E73E0F72E01E02FE130E0C0
:105BE0004FEF5FEF62E370E08FE090E00E94990575
:105BF000E6E0EE2EE3E0FE2E2FE130E04FEF5FEF28
:105C000066E470E08FE090E00E949905E090120653
:105C1000F090130603E02FE130E04FEF5FEF62E812
:105C200070E080E590E00E94DF0580912D06909164
:105C30002E068130910531F4809184068F5F809328
:105C4000840639C00297B9F5809112069091130627
:105C50008636910520F010921306109212065EE12E
:105C6000E52E53E0F52E01E02FE130E04FEF5FEF3E
:105C700062E370E08FE090E00E94990566E0E62E16
:105C800063E0F62E2FE130E04FEF5FEF66E470E067
:105C90008FE090E00E949905E0901206F0901306C4
:105CA00003E02FE130E04FEF5FEF62E870E080E566
:105CB00090E00E94DF0580912D0690912E060497BA
:105CC000B9F580911206909113068636910520F061
:105CD00010921306109212063EE1E32E33E0F32EEB
:105CE00001E02FE130E04FEF5FEF62E370E08FE023
:105CF00090E00E94990546E0E42E43E0F42E2FE167
:105D000030E04FEF5FEF66E470E08FE090E00E94DC
:105D10009905E0901206F090130603E02FE130E0C1
:105D20004FEF5FEF62E870E080E590E00E94DF05F2
:105D300080912D0690912E060597B9F58091120657
:105D4000909113068636910520F01092130610925A
:105D500012069EE1E92E93E0F92E01E02FE130E0FA
:105D60004FEF5FEF62E370E08FE090E00E949905F3
:105D700026E0E22E23E0F22E2FE130E04FEF5FEF3E
:105D800066E470E08FE090E00E949905E0901206D2
:105D9000F090130603E02FE130E04FEF5FEF62E891
:105DA00070E080E590E00E94DF0580912D069091E3
:105DB0002E06069709F0E8C180911206909113060D
:105DC0008636910520F010921306109212061EE1FD
:105DD000E12E13E0F12E01E02FE130E04FEF5FEF15
:105DE00062E370E08FE090E00E94990586E0E82E83
:105DF00083E0F82E2FE130E04FEF5FEF66E470E0D4
:105E00008FE090E00E949905E0901206F090130652
:105E100003E02FE130E04FEF5FEF62E870E080E5F4
:105E200090E00E94DF05B0C1892B49F580911C06E6
:105E300090911D068D32914020F010921D06109217
:105E40001C06B6E8EB2EB2E0FB2E01E02FE130E0BD
:105E50004FEF5FEF6CE370E08FE090E00E949905F8
:105E6000E0901C06F0901D0603E02FE130E04FEFBC
:105E70005FEF62E870E080E590E00E94DF058091CE
:105E80002D0690912E06019709F079C080911C068D
:105E900090911D068D32914020F010921D061092B7
:105EA0001C06A6E8EA2EA2E0FA2E01E02FE130E07F
:105EB0004FEF5FEF6CE370E08FE090E00E94990598
:105EC000E0901C06F0901D064FC0892B49F580918B
:105ED0001E0690911F06893E934020F010921F06E7
:105EE00010921E06FCEDEF2EF2E0FF2E01E02FE1F6
:105EF00030E04FEF5FEF6CE370E08FE090E00E94E6
:105F00009905E0901E06F0901F0603E02FE130E0B7
:105F10004FEF5FEF62E870E080E590E00E94DF0500
:105F200080912D0690912E06019749F580911E06CD
:105F300090911F06893E934020F010921F06109208
:105F40001E06ECEDEE2EE2E0FE2E01E02FE130E049
:105F50004FEF5FEF6CE370E08FE090E00E949905F7
:105F6000E0901E06F0901F0603E02FE130E04FEFB7
:105F70005FEF62E870E080E590E00E94DF058091CD
:105F80002D0690912E068230910509F4B8C09C012F
:105F9000245031092230310508F0AEC0B0C0892B41
:105FA00009F094C08091140690911506039720F093
:105FB000109215061092140674EFE72E72E0F72E79
:105FC00001E02FE130E04FEF5FEF6CE370E08EE136
:105FD00090E00E9499058091140690911506019712
:105FE00079F463E5E62E65E0F62E03E02FE130E07C
:105FF0004FEF5FEF62E870E080E590E00E94990566
:106000008091140690911506892B79F45EE4E52EB3
:1060100055E0F52E03E02FE130E04FEF5FEF62E84F
:1060200070E080E590E00E949905809114068093CD
:10603000F4054CC0892B09F049C08091F405811109
:106040000BC01092840653C0892B09F03FC0809189
:10605000F405811149C0F5CF813009F048C0809125
:10606000160690911706893E934020F0109217066D
:10607000109216063EE7E32E33E0F32E01E02FE107
:1060800030E04FEF5FEF62E370E08FE090E00E945E
:10609000990546ECE42E42E0F42E2FE130E04FEF7C
:1060A0005FEF66E470E08FE090E00E949905E09079
:1060B0001606F090170603E02FE130E04FEF5FEF98
:1060C00062E870E080E590E00E94DF0580912D0697
:1060D00090912E068130910591F08230910579F0F2
:1060E0008430910561F005C0813009F47DC180E004
:1060F00090E08530910519F0069709F045C0809130
:1061000084068F5F809384063FC0009731F09C0126
:10611000215031092230310518F4109284062BC029
:10612000049749F58091200690912106893E93407D
:1061300020F010922106109220068FE5E82E82E0D2
:10614000F82E01E02FE130E04FEF5FEF6CE370E0FD
:106150008FE090E00E949905E0902006F0902106E3
:1061600003E02FE130E04FEF5FEF62E870E080E5A1
:1061700090E00E94DF0580912D0690912E060597F4
:10618000029710F41092840680915306813009F032
:106190000EC1809398061092600680912D06909112
:1061A0002E06892B41F5E0913806F0913906E8304A
:1061B000F10508F5EB57FF4F4EE150E00C94CD444C
:1061C00064E972E014C066E772E011C068E572E04D
:1061D0000EC06AE372E00BC06CE172E008C06EEFC3
:1061E00071E005C060EE71E002C062EC71E084E035
:1061F00096E00E94F54780912D0690912E0601971A
:10620000E1F480913806909139068130910569F06A
:1062100038F0029791F44EE150E068E671E009C071
:106220004EE150E064EA71E004C04EE150E066E8FF
:1062300071E084E096E00E94F54780912D069091F0
:106240002E060297E1F4809138069091390681304C
:10625000910569F038F0029791F44EE150E06EE05C
:1062600071E009C04EE150E06AE471E004C04EE123
:1062700050E06CE271E084E096E00E94F547809186
:106280002D0690912E060497E1F4809138069091A6
:1062900039068130910569F038F0029791F44EE1AA
:1062A00050E064EB70E009C04EE150E060EF70E058
:1062B00004C04EE150E062ED70E084E096E00E94A0
:1062C000F54780912D0690912E060597E1F4809177
:1062D0003806909139068130910569F038F00297BF
:1062E00091F44EE150E06AE570E009C04EE150E003
:1062F00066E970E004C04EE150E068E770E084E0D9
:1063000096E00E94F54780912D0690912E06069703
:10631000E1F480913806909139068130910569F059
:1063200038F0029791F44EE150E060E070E009C06F
:106330004EE150E06CE370E004C04EE150E06EE1ED
:1063400070E084E096E00E94F5478FE190E00E94C3
:10635000190680912D0690912E06892B09F47FD184
:1063600080912D0690912E06019711F40E94CB3B4F
:1063700080912D0690912E06029711F40E94D23C36
:1063800080912D0690912E06049711F40E94D93D1C
:1063900080912D0690912E06059711F40E941726E4
:1063A00080912D0690912E06069709F450D0809189
:1063B000530681110CC081E080939806109260060C
:1063C000109222068FE190E00E941906EBD2C09352
:1063D00053068FE798E321E0815090402040E1F799
:1063E00000C000000C943127809118069091190686
:1063F000893E934020F010921906109218069FEAE9
:10640000E92E92E0F92E01E02FE130E04FEF5FEF4F
:1064100062E370E08FE090E00E9499052CE9E22EA3
:1064200022E0F22E2FE130E04FEF5FEF66E470E004
:106430008FE090E00E949905E0901806F090190610
:106440003ACECF911F910F91FF90EF900895EF9268
:10645000FF920F931F93CF93DF93A89580916006CF
:106460008111F6C08FE190E00E9419060E944F0C46
:106470008091860690E0909339068093380685E0F7
:1064800080935306C1E0D5E0809160068111E0C0A1
:10649000A8950E94DD0C809153068230A9F480916A
:1064A0003806909139060196909339068093380604
:1064B0000FE110E02CE330E046EE50E069E670E0DA
:1064C00081E090E00E94A404809153068330A9F4F7
:1064D0008091380690913906019790933906809300
:1064E00038060FE110E02CE330E046EE50E069E6BC
:1064F00070E081E090E00E94A404809138069091C1
:106500003906039720F010923906109238068091D0
:106510003806909139068130910589F1D0F00297C3
:1065200009F046C081E8E82E84E0F82E02E02FE171
:1065300030E04FEF5FEF6DE770E088E290E00E949F
:10654000990582E0809386064EE150E060E070E0BD
:106550002BC025E9E22E24E0F22E02E02FE130E00C
:106560004FEF5FEF6DE770E088E290E00E949905E1
:10657000109286064EE150E06CE370E015C09BE897
:10658000E92E94E0F92E02E02FE130E04FEF5FEFCB
:106590006DE770E088E290E00E949905C09386065E
:1065A0004EE150E06EE170E084E096E00E94D84752
:1065B00080915306811110C0A895C0936006109277
:1065C0003F0610923E06C0934E068FE190E00E9477
:1065D0001906A8950E94E91F80915306813061F544
:1065E000A8958093600610923F0610923E06809315
:1065F0004E068FE190E00E941906A8951092980629
:1066000080918606813069F038F0823091F44EE155
:1066100050E060E070E009C04EE150E06CE370E0F3
:1066200004C04EE150E06EE170E084E096E00E942C
:10663000D847A8950E941D27D09353062FEF80E7D7
:1066400092E0215080409040E1F700C000001CCF54
:10665000DF91CF911F910F91FF90EF900895AF922E
:10666000BF92CF92DF92EF92FF920F931F93CF933F
:10667000DF93A89580916006811189C18FE190E038
:106680000E9419060E944F0C80918A0690E0909318
:1066900039068093380685E080935306E7E0DE2EC6
:1066A000F6E0CF2ED5E0A4E0BA2EB3E0AB2EC1E0E9
:1066B0008091600681116BC1A8950E94DD0C8091CC
:1066C00053068230A9F480913806909139060196DC
:1066D00090933906809338060FE110E02CE330E008
:1066E00046EE50E069E670E081E090E00E94A4048C
:1066F000809153068330A9F4809138069091390631
:10670000019790933906809338060FE110E02CE34F
:1067100030E046EE50E069E670E081E090E00E94F3
:10672000A4048091380690913906089720F01092C1
:10673000390610923806E0913806F0913906E830B3
:10674000F10508F0BEC0E357FF4F0C94CD4474EA46
:10675000E72E74E0F72E02E02FE130E04FEF5FEF1D
:106760006DE770E082E390E00E94990510928A063E
:106770004EE150E064E972E09AC06FE9E62E64E011
:10678000F62E02E02FE130E04FEF5FEF6DE770E0B3
:1067900082E390E00E949905C0938A064EE150E0A2
:1067A00066E772E084C055E9E52E54E0F52E02E07C
:1067B0002FE130E04FEF5FEF6DE770E088E290E0AF
:1067C0000E94990582E080938A064EE150E068E5D8
:1067D00072E06DC04BE8E42E44E0F42E02E02FE1BD
:1067E00030E04FEF5FEF6DE770E088E290E00E94ED
:1067F0009905A0928A064EE150E06AE372E057C024
:1068000031E8E32E34E0F32E02E02FE130E04FEFE9
:106810005FEF6DE770E088E290E00E949905B0922A
:106820008A0644E150E06CE172E041C027E7E22EC5
:1068300024E0F22E02E02FE130E04FEF5FEF6DE752
:1068400070E088E290E00E949905D0938A064EE1BC
:1068500050E06EEF71E02BC09DE6E92E94E0F92E3A
:1068600002E02FE130E04FEF5FEF6DE770E088E28C
:1068700090E00E949905C0928A064EE150E060EED9
:1068800071E015C083E6E82E84E0F82E02E02FE1E7
:1068900030E04FEF5FEF6DE770E088E290E00E943C
:1068A0009905D0928A064EE150E062EC71E084E0F6
:1068B00096E00E94D8478FE59AEE0197F1F700C065
:1068C00000008091530681110FC0A895C093600607
:1068D00010923F0610923E06C0934E068FE190E064
:1068E0000E9419060E94E91F80915306813009F029
:1068F00041C0A8958093600610923F0610923E0614
:1069000080934E068FE190E00E941906109298063F
:10691000E0918A068E2F90E08830910540F5FC01C9
:10692000EB56FF4F4EE150E00C94CD4464E972E029
:1069300014C066E772E011C068E572E00EC06AE359
:1069400072E00BC06CE172E008C06EEF71E005C050
:1069500060EE71E002C062EC71E084E096E00E94BB
:10696000D8478FE59AEE0197F1F700C00000A8958F
:106970000E941D27D0935306A8959FEF20E782E041
:10698000915020408040E1F700C0000091CEDF919F
:10699000CF911F910F91FF90EF90DF90CF90BF901C
:1069A000AF900895BF92CF92DF92EF92FF920F9334
:1069B0001F93CF93DF93809122068111E2C68FE16E
:1069C00090E00E9419060E94450D1092850685E010
:1069D0008093530698E5C92E92E0D92ECAE5D0E0FF
:1069E00025E0B22E809122068111CBC6E09184066B
:1069F0008E2F90E08E30910508F0B2C6FC01E35670
:106A0000FF4F0C94CD441BE3E12E14E0F12E01E086
:106A10002FE130E04FEF5FEF62E370E08FE090E056
:106A20000E94990584E3E82E84E0F82E2FE130E0FF
:106A30004FEF5FEF66E470E08CE390E00E94990511
:106A4000E0900406F090050603E02FE130E040E01E
:106A500058EF62E870E080E590E00E94DF058091E9
:106A60000406909105069093F9058093F8050E941D
:106A7000DD0C809153068230A9F48091F805909145
:106A8000F90501969093F9058093F8050FE110E060
:106A90002CE330E046EE50E069E670E081E090E003
:106AA0000E94A404809153068330A9F48091F805D4
:106AB0009091F90501979093F9058093F8050FE1FE
:106AC00010E02CE330E046EE50E069E670E081E053
:106AD00090E00E94A4048091F8059091F9058F350B
:106AE000914020F01092F9051092F8058091F80578
:106AF0009091F905909305068093040628C6ACE1B1
:106B0000EA2EA4E0FA2E01E02FE130E04FEF5FEF34
:106B100062E370E08FE090E00E949905BEE0EB2E0A
:106B2000B4E0FB2E2FE130E04FEF5FEF66E470E062
:106B30008CE390E00E949905E0900606F09007062D
:106B400003E02FE130E040E058EF62E870E080E5DC
:106B500090E00E94DF0580910606909107069093D1
:106B60004B0680934A060E94DD0C809153068230CA
:106B7000A9F480914A0690914B06019690934B069A
:106B800080934A060FE110E02CE330E046EE50E03F
:106B900069E670E081E090E00E94A40480915306D1
:106BA0008330A9F480914A0690914B060197909307
:106BB0004B0680934A060FE110E02CE330E046EEEE
:106BC00050E069E670E081E090E00E94A4048091CA
:106BD0004A0690914B06853F914020F010924B065B
:106BE00010924A0680914A0690914B0690930706B0
:106BF00080930606ACC5E6EFEE2EE3E0FE2E01E044
:106C00002FE130E04FEF5FEF62E370E08FE090E064
:106C10000E949905FEEDEF2EF3E0FF2E2FE130E00C
:106C20004FEF5FEF66E470E08FE090E00E9499051F
:106C3000E0900806F090090603E02FE130E040E024
:106C400058EF62E870E080E590E00E94DF058091F7
:106C500008069091090690939306809392060E94ED
:106C6000DD0C809153068230A9F4809192069091B8
:106C70009306019690939306809392060FE110E09D
:106C80002CE330E046EE50E069E670E081E090E011
:106C90000E94A404809153068330A9F48091920647
:106CA00090919306019790939306809392060FE13B
:106CB00010E02CE330E046EE50E069E670E081E061
:106CC00090E00E94A40480919206909193064F97C1
:106CD00030F08FE090E0909393068093920680913D
:106CE0009206909193060F9730F48FE090E0909386
:106CF00093068093920680919206909193069093CA
:106D000009068093080623C566ECE62E63E0F62E9E
:106D100001E02FE130E04FEF5FEF62E370E08FE0E2
:106D200090E00E9499057EEAE72E73E0F72E2FE1AE
:106D300030E04FEF5FEF66E470E08FE090E00E949C
:106D40009905E0900A06F0900B0603E02FE130E091
:106D500040E058EF62E870E080E590E00E94DF05D7
:106D600080910A0690910B06909335068093340625
:106D70000E94DD0C809153068230A9F48091340684
:106D800090913506019690933506809334060FE175
:106D900010E02CE330E046EE50E069E670E081E080
:106DA00090E00E94A404809153068330A9F480915E
:106DB00034069091350601979093350680933406FA
:106DC0000FE110E02CE330E046EE50E069E670E0C1
:106DD00081E090E00E94A4048091340690913506F1
:106DE0004F9730F08FE090E0909335068093340613
:106DF00080913406909135060F9730F48FE090E043
:106E00009093350680933406809134069091350630
:106E100090930B0680930A069AC456E9E52E53E038
:106E2000F52E01E02FE130E04FEF5FEF6CE370E013
:106E30008FE090E00E94990580910C0690910D06DC
:106E4000019779F443E5E42E45E0F42E03E02FE1C9
:106E500030E040E058EF62E870E080E590E00E94AA
:106E6000990580910C0690910D06892B79F43EE4EA
:106E7000E32E35E0F32E03E02FE130E040E058EF61
:106E800062E870E080E590E00E94990580910C0630
:106E900080935F060E94DD0C80915306823089F456
:106EA00080915F068F5F80935F060FE110E02CE317
:106EB00030E046EE50E069E670E081E090E00E944C
:106EC000A40480915306833089F480915F06815039
:106ED00080935F060FE110E02CE330E046EE50E0D7
:106EE00069E670E081E090E00E94A40480915F0672
:106EF000823010F010925F0680915F0690E09093D0
:106F00000D0680930C0623C49EE7E92E93E0F92E2C
:106F100001E02FE130E04FEF5FEF62E370E08FE0E0
:106F200090E00E94990526E6E22E23E0F22E2FE162
:106F300030E04FEF5FEF66E470E08FE090E00E949A
:106F40009905E0900E06F0900F0603E020E038EF80
:106F50004FEF5FEF62E870E080E590E00E94DF05B0
:106F600080910E0690910F0690933306809332061F
:106F70000E94DD0C809153068230A9F48091320684
:106F800090913306019690933306809332060FE179
:106F900010E02CE330E046EE50E069E670E081E07E
:106FA00090E00E94A404809153068330A9F480915C
:106FB0003206909133060197909333068093320600
:106FC0000FE110E02CE330E046EE50E069E670E0BF
:106FD00081E090E00E94A4048091320690913306F3
:106FE0008B3F910520F0109233061092320680916B
:106FF00032069091330690930F0680930E06A7C336
:107000001EE4E12E13E0F12E01E02FE130E04FEF1E
:107010005FEF62E370E08FE090E00E94990586E305
:10702000E82E83E0F82E2FE130E04FEF5FEF66E4CB
:1070300070E08FE090E00E949905E0901006F090DB
:10704000110603E02FE130E040E058EF62E870E025
:1070500080E590E00E94DF05809110068093430652
:107060000E94DD0C80915306823089F480914306A2
:107070008F5F809343060FE110E02CE330E046EE93
:1070800050E069E670E081E090E00E94A404809105
:107090005306833089F480914306815080934306E0
:1070A0000FE110E02CE330E046EE50E069E670E0DE
:1070B00081E090E00E94A40480914306853610F0A0
:1070C000109243068091430690E0909311068093BE
:1070D00010063DC3AEE1EA2EA3E0FA2E01E02FE157
:1070E00030E04FEF5FEF62E370E08FE090E00E94EE
:1070F0009905B6E0EB2EB3E0FB2E2FE130E04FEF29
:107100005FEF66E470E08FE090E00E949905E09008
:107110001206F090130603E02FE130E040E058EF54
:1071200062E870E080E590E00E94DF058091120641
:10713000809342060E94DD0C80915306823089F4D0
:10714000809142068F5F809342060FE110E02CE3AE
:1071500030E046EE50E069E670E081E090E00E94A9
:10716000A40480915306833089F4809142068150B3
:10717000809342060FE110E02CE330E046EE50E051
:1071800069E670E081E090E00E94A40480914206EC
:10719000853610F0109242068091420690E090935E
:1071A000130680931206D3C2F6E8EF2EF2E0FF2E0C
:1071B00001E02FE130E04FEF5FEF6CE370E08FE034
:1071C00090E00E949905E0901C06F0901D0603E0F7
:1071D0002FE130E040E058EF62E870E080E590E0B9
:1071E0000E94DF0580911C0690911D0690938106F8
:1071F000809380060E94DD0C809153068230A9F4B2
:1072000080918006909181060196909381068093EB
:1072100080060FE110E02CE330E046EE50E069E636
:1072200070E081E090E00E94A404809153068330D6
:10723000A9F4809180069091810601979093810630
:10724000809380060FE110E02CE330E046EE50E042
:1072500069E670E081E090E00E94A40480918006DD
:1072600090918106893C910520F0D0938106C093CE
:10727000800680918006909181068A35910520F4E0
:10728000D0938106C09380068091800690918106FC
:1072900090931D0680931C065AC2ECEDEE2EE2E0A0
:1072A000FE2E01E02FE130E04FEF5FEF6CE370E086
:1072B0008FE090E00E949905E0901E06F0901F0676
:1072C00003E02FE130E040E058EF62E870E080E555
:1072D00090E00E94DF0580911E0690911F0690931A
:1072E0000306809302060E94DD0C809153068230D3
:1072F000A9F48091020690910306019690930306EB
:10730000809302060FE110E02CE330E046EE50E0FF
:1073100069E670E081E090E00E94A4048091530649
:107320008330A9F48091020690910306019790930F
:107330000306809302060FE110E02CE330E046EEF6
:1073400050E069E670E081E090E00E94A404809142
:10735000020690910306C39720F010920306109244
:107360000206809102069091030690931F06809377
:107370001E06EDC174EFE72E72E0F72E01E02FE15B
:1073800030E04FEF5FEF6CE370E08EE190E00E9441
:1073900099058091140690911506019779F463E59B
:1073A000E62E65E0F62E03E02FE130E040E058EFF6
:1073B00062E870E080E590E00E94990580911406F3
:1073C00090911506892B79F45EE4E52E55E0F52EB3
:1073D00003E02FE130E040E058EF62E870E080E544
:1073E00090E00E949905809114068093F4050E9414
:1073F000DD0C80915306823089F48091F4058F5F13
:107400008093F4050FE110E02CE330E046EE50E00D
:1074100069E670E081E090E00E94A4048091530648
:10742000833089F48091F40581508093F4050FE155
:1074300010E02CE330E046EE50E069E670E081E0D9
:1074400090E00E94A4048091F405823010F0109224
:10745000F4058091F40590E090931506809314064E
:1074600076C18091F405811103C01092840678C121
:10747000813009F075C13EE7E32E33E0F32E01E0E1
:107480002FE130E04FEF5FEF62E370E08FE090E0DC
:107490000E94990546ECE42E42E0F42E2FE130E004
:1074A0004FEF5FEF66E470E08FE090E00E94990597
:1074B000E0901606F090170603E02FE130E040E080
:1074C00058EF62E870E080E590E00E94DF0580916F
:1074D00016069091170690938306809382060E9469
:1074E000DD0C809153068230A9F480918206909140
:1074F0008306019690938306809382060FE110E045
:107500002CE330E046EE50E069E670E081E090E088
:107510000E94A404809153068330A9F480918206CE
:1075200090918306019790938306809382060FE1E2
:1075300010E02CE330E046EE50E069E670E081E0D8
:1075400090E00E94A40480918206909183068B3F74
:10755000910520F010928306109282068091820697
:10756000909183069093170680931606F0C0809141
:10757000F405882309F479CF813009F0F1C09FEA3E
:10758000E92E92E0F92E01E02FE130E04FEF5FEFBE
:1075900062E370E08FE090E00E9499052CE9E22E12
:1075A00022E0F22E2FE130E04FEF5FEF66E470E073
:1075B0008FE090E00E949905E0901806F09019067F
:1075C00003E02FE130E040E058EF62E870E080E552
:1075D00090E00E94DF058091180690911906909323
:1075E0005E0680935D060E94DD0C8091530682301A
:1075F000A9F480915D0690915E06019690935E06D7
:1076000080935D060FE110E02CE330E046EE50E0A1
:1076100069E670E081E090E00E94A4048091530646
:107620008330A9F480915D0690915E060197909356
:107630005E0680935D060FE110E02CE330E046EE3D
:1076400050E069E670E081E090E00E94A40480913F
:107650005D0690915E06C39720F010925E06109230
:107660005D0680915D0690915E0690931906809369
:1076700018066DC08FE5E82E82E0F82E01E02FE1BC
:1076800030E04FEF5FEF6CE370E08FE090E00E943E
:107690009905E0902006F090210603E02FE130E00C
:1076A00040E058EF62E870E080E590E00E94DF057E
:1076B00080912006909121069093280680932706BA
:1076C0000E94DD0C809153068230A9F48091270638
:1076D00090912806019690932806809327060FE143
:1076E00010E02CE330E046EE50E069E670E081E027
:1076F00090E00E94A404809153068330A9F4809105
:1077000027069091280601979093280680932706D4
:107710000FE110E02CE330E046EE50E069E670E067
:1077200081E090E00E94A4048091020690910306FB
:107730008935924020F0D0922806C0922706809189
:1077400027069091280690932106809320068FE7C4
:1077500098E321E0815090402040E1F700C0000014
:1077600080915306813051F480932206109298063E
:107770008FE190E00E9419060E941D27B0925306E7
:1077800031C9DF91CF911F910F91FF90EF90DF9062
:10779000CF90BF900895EF92FF920F931F93CF93D6
:1077A000DF93A895809160068111F5C08FE190E08C
:1077B0000E9419060E944F0C8091360690E090932B
:1077C00039068093380685E080935306C1E0D5E002
:1077D000809160068111DFC0A8950E94DD0C809128
:1077E00053068230A9F480913806909139060196AB
:1077F00090933906809338060FE110E02CE330E0D7
:1078000046EE50E069E670E081E090E00E94A4045A
:10781000809153068330A9F48091380690913906FF
:10782000019790933906809338060FE110E02CE31E
:1078300030E046EE50E069E670E081E090E00E94C2
:10784000A4048091380690913906039720F0109295
:10785000390610923806A89580913806909139061D
:107860008130910589F1D0F0029709F046C081E896
:10787000E82E84E0F82E02E02FE130E04FEF5FEFDA
:107880006DE770E088E290E00E94990582E08093C5
:1078900036064EE150E068E671E02BC025E9E22EA5
:1078A00024E0F22E02E02FE130E04FEF5FEF6DE7D2
:1078B00070E088E290E00E949905109236064EE151
:1078C00050E064EA71E015C09BE8E92E94E0F92EDF
:1078D00002E02FE130E04FEF5FEF6DE770E088E20C
:1078E00090E00E949905C09336064EE150E066E8AC
:1078F00071E084E096E00E94D847809153068111A0
:107900000FC0A895C093600610923F0610923E06E5
:10791000C0934E068FE190E00E9419060E94E91F75
:1079200080915306813059F5A89580936006109296
:107930003F0610923E0680934E068FE190E00E9433
:1079400019061092980680913606813069F038F059
:10795000823091F44EE150E068E671E009C04EE1FA
:1079600050E064EA71E004C04EE150E066E871E086
:1079700084E096E00E94D847A8950E941D27D093E6
:1079800053062FEF80E792E0215080409040E1F7CE
:1079900000C000001DCFDF91CF911F910F91FF908C
:1079A000EF900895EF92FF920F931F93CF93DF9381
:1079B000A895809160068111F5C08FE190E00E944A
:1079C00019060E944F0C80913D0690E09093390675
:1079D0008093380685E080935306C1E0D5E080911E
:1079E00060068111DFC0A8950E94DD0C80915306CE
:1079F0008230A9F4809138069091390601969093CF
:107A00003906809338060FE110E02CE330E046EEB3
:107A100050E069E670E081E090E00E94A40480916B
:107A200053068330A9F48091380690913906019766
:107A300090933906809338060FE110E02CE330E094
:107A400046EE50E069E670E081E090E00E94A40418
:107A50008091380690913906039720F010923906EC
:107A60001092380680913806909139068130910540
:107A700089F1D0F0029709F046C081E8E82E84E051
:107A8000F82E02E02FE130E04FEF5FEF6DE770E09E
:107A900088E290E00E94990582E080933D064EE1E5
:107AA00050E06EE071E02BC025E9E22E24E0F22EDA
:107AB00002E02FE130E04FEF5FEF6DE770E088E22A
:107AC00090E00E94990510923D064EE150E06AE474
:107AD00071E015C09BE8E92E94E0F92E02E02FE159
:107AE00030E04FEF5FEF6DE770E088E290E00E94DA
:107AF0009905C0933D064EE150E06CE271E084E0F0
:107B000096E00E94D84780915306811110C0A89535
:107B1000C093600610923F0610923E06C0934E0638
:107B20008FE190E00E941906A8950E94E91F8091BC
:107B30005306813059F5A8958093600610923F0650
:107B400010923E0680934E068FE190E00E94190647
:107B50001092980680913D06813069F038F08230AD
:107B600091F44EE150E06EE071E009C04EE150E06A
:107B70006AE471E004C04EE150E06CE271E084E040
:107B800096E00E94D847A8950E941D27D0935306DF
:107B90002FEF80E792E0215080409040E1F700C055
:107BA00000001DCFDF91CF911F910F91FF90EF90BB
:107BB0000895EF92FF920F931F93CF93DF93A895B1
:107BC000809160068111F6C08FE190E00E94190655
:107BD0000E944F0C8091950690E090933906809317
:107BE000380685E080935306C1E0D5E080916006B9
:107BF0008111E0C0A8950E94DD0C8091530682306F
:107C0000A9F480913806909139060196909339062F
:107C1000809338060FE110E02CE330E046EE50E0B0
:107C200069E670E081E090E00E94A4048091530630
:107C30008330A9F48091380690913906019790938A
:107C40003906809338060FE110E02CE330E046EE71
:107C500050E069E670E081E090E00E94A404809129
:107C6000380690913906039720F010923906109249
:107C7000380680913806909139068130910589F156
:107C8000D0F0029709F046C081E8E82E84E0F82E93
:107C900002E02FE130E04FEF5FEF6DE770E088E248
:107CA00090E00E94990582E0809395064EE150E0B5
:107CB00064EB70E02BC025E9E22E24E0F22E02E016
:107CC0002FE130E04FEF5FEF6DE770E088E290E08A
:107CD0000E949905109295064EE150E060EF70E029
:107CE00015C09BE8E92E94E0F92E02E02FE130E088
:107CF0004FEF5FEF6DE770E088E290E00E9499053A
:107D0000C09395064EE150E062ED70E084E096E0AD
:107D10000E94D84780915306811110C0A895C09346
:107D2000600610923F0610923E06C0934E068FE109
:107D300090E00E941906A8950E94E91F80915306C1
:107D4000813061F5A8958093600610923F061092ED
:107D50003E0680934E068FE190E00E941906A8959A
:107D60001092980680919506813069F038F0823043
:107D700091F44EE150E064EB70E009C04EE150E058
:107D800060EF70E004C04EE150E062ED70E084E02E
:107D900096E00E94D847A8950E941D27D0935306CD
:107DA0002FEF80E792E0215080409040E1F700C043
:107DB00000001CCFDF91CF911F910F91FF90EF90AA
:107DC00008950F931F9380912B0690912C06892B79
:107DD00009F09EC080918C0690918D0683359105A7
:107DE000A9F581E090E090932C0680932B060E94E9
:107DF00029140FE110E02CE330E044E650E06BE49E
:107E000070E08EE690E00E94A40424E230E04AE5AF
:107E100050E064E670E088E090E00E94A40424E270
:107E200030E04AE550E064E670E088E090E00E94CF
:107E3000A40424E230E04AE550E064E670E08FED0F
:107E400090E00E94A4040E94E91FA8950E94BE1E13
:107E50000E949F1AA89503E02FE130E04FEF5FEFFB
:107E600069E170E085E890E00E9404110E946C1EB8
:107E70000E949C1080912B0690912C060197A9F5E9
:107E8000A8950E9429140FE110E02CE330E044E6AD
:107E900050E06BE470E08EE690E00E94A40424E2DF
:107EA00030E04AE550E064E670E088E090E00E944F
:107EB000A40424E230E04AE550E064E670E088E0A3
:107EC00090E00E94A40424E230E04AE550E064E639
:107ED00070E08FED90E00E94A4048091F305813062
:107EE00009F4D2D10E94E91FA8952FEF81EE94E00A
:107EF000215080409040E1F700C000000E94D20E67
:107F00000E94951E0E94580F1F910F910C94C80F4C
:107F10001F910F9108951F920F920FB60F92112487
:107F20008F939F938CB190E090938D0680938C06F5
:107F30009F918F910F900FBE0F901F9018951F92D9
:107F40000F920FB60F9211242F938F939F938091CE
:107F5000FE059091FF050196883E23E0920728F4E4
:107F60009093FF058093FE0504C01092FF051092C8
:107F7000FE0580912906811105C010928F0610928E
:107F80008E060BC0813049F480918E0690918F0649
:107F9000019690938F0680938E06809148068111FA
:107FA00005C01092FD051092FC050BC0813049F40C
:107FB0008091FC059091FD0501969093FD058093BD
:107FC000FC0580914006811105C0109201061092B7
:107FD00000060BC0813049F48091000690910106A3
:107FE000019690930106809300069F918F912F91A7
:107FF0000F900FBE0F901F9018952FEF89E698E114
:10800000215080409040E1F700C000008FEF8ABB14
:1080100081BB8093610081E084BB88EA8FBD8CE0E6
:108020008EBD1DBC1CBC17BC16BC8AE78BBD82E193
:108030008ABD19BC18BC109279001092780080E1BA
:1080400087BF10BE87E683BF12BE11BE81E8809352
:108050008B0085E080938A0010928900109288003E
:10806000109281001092800010928700109286007A
:10807000109285001092840010928300109282006A
:108080001BB888E98AB986E0809395001092900029
:108090008FE289B98FE181BD8FE081BDCED281E0D1
:1080A0000E94B0038FE190E00E94190681E090E009
:1080B00090932C0680932B0610923F0610923E065A
:1080C00010922E0610922D061092FF051092FE05BA
:1080D00010924506109244061092FB0510922A0653
:1080E000109290061092230680E590E090938D0602
:1080F00080938C06809164008E7F809364008091D1
:108100006500816080936500809164008860809341
:108110006400809165008860809365001092F3058B
:108120007894A49AAC9A2FEF85EA9EE02150804083
:108130009040E1F700C00000A895AC9882EB92E077
:1081400047D7813011F4A8950FC00E94DE1AA89578
:108150000E944B1EA89561E083EB92E04FD7A89553
:1081600061E082EB92E04AD7A89580912B0690912E
:108170002C06019721F4A8950E94E91FA895A895BF
:1081800020DEF2CF80916400806180936400809152
:1081900065008061809365008091640088608093B1
:1081A000640080916500877F809365008091EE0573
:1081B0009091EF058536910500F58091640084600B
:1081C00080936400809165008460809365008FECEB
:1081D00097E00197F1F700C00000A8958091650035
:1081E0008B7F809365008091EE059091EF0501965D
:1081F0009093EF058093EE05D9CF8091650088605C
:10820000809365000895809164008061809364008C
:10821000809165008F7E8093650080916400886006
:108220008093640080916500877F809365008091D2
:10823000EE059091EF058536910500F5809164007B
:108240008460809364008091650084608093650001
:108250008FEC97E00197F1F700C00000A89580919E
:1082600065008B7F809365008091EE059091EF050E
:1082700001969093EF058093EE05D9CF809165002C
:1082800088608093650008958AEB92E0A1D6809380
:108290009A068091640080618093640080916500FB
:1082A00080618093650080916400886080936400A1
:1082B00080916500877F8093650080919A0624E60F
:1082C000829FC00111242091EC053091ED05281703
:1082D000390700F580916400846080936400809188
:1082E00065008460809365008FEC97E00197F1F75B
:1082F00000C00000A895809165008B7F8093650089
:108300008091EC059091ED0501969093ED05809399
:10831000EC05D3CF80916500886080936500109252
:10832000F2051092ED051092EC050895AC018091D4
:10833000F20581114AC090916400906190936400AD
:10834000909165009F7E9093650090916400986085
:108350009093640090916500977F9093650084E608
:10836000849F9001859F300D11248091EC059091A0
:10837000ED058217930700F5809164008460809377
:108380006400809165008460809365008FEC97E0C5
:108390000197F1F700C00000A895809165008B7FE0
:1083A000809365008091EC059091ED050196909386
:1083B000ED058093EC05D9CF8091650088608093AE
:1083C00065001092ED051092EC0581E08093F205B6
:1083D0000895682F8AEB92E011C68AEB92E0F8D5F7
:1083E00090E0A4CF8093F1050895CF93DF9300D060
:1083F00000D0CDB7DEB7809163001C821B821A8249
:108400001982BE016F5F7F4FCE01039629D18B8108
:108410009C818431954068F489819A81843A9640A0
:1084200040F489819A818D32914018F082E08093E6
:108430009C068B819C818937954090F08B819C8133
:10844000843C994068F489819A81843A964040F44A
:1084500089819A818D32914018F083E080939C0647
:108460008B819C8189329A4068F089819A81843716
:108470009E4040F489819A81813D974018F081E0C7
:1084800080939C068B819C81863F994060F48B8110
:108490009C818134964038F089819A81813D974052
:1084A00010F010929C0680919C060F900F900F90F8
:1084B0000F90DF91CF910895DF92EF92FF920F938B
:1084C0001F93CF93DF9385E080939C06DBE485E0E8
:1084D000D82E8091F10581116FC087DFE090F00503
:1084E000F12C03E02FE130E040E058EF62E870E06B
:1084F00080E590E00E94DF0580919C068230B1F417
:108500008091F00581508093F0051092EF05109254
:10851000EE050FE110E02CE330E046EE50E069E6B6
:1085200070E081E090E00E94A4042CDE80919C0623
:108530008330C1F48091F0058B34A0F48F5F809379
:10854000F0051092EF051092EE050FE110E02CE31C
:1085500030E046EE50E069E670E081E090E00E9495
:10856000A40451DE8091F0058C3410F0D093F00516
:1085700080919C0681110EC00FE110E02CE330E0E9
:1085800046EE50E069E670E081E090E00E94A404CD
:108590001092F005C0919C06C13059F48091F0050D
:1085A00018DF8091F00590E06FDE1092F005C09327
:1085B000F105D0929C068DCFDF91CF911F910F9145
:1085C000FF90EF90DF900895EF92FF920F938AEB68
:1085D00092E0FED4E82EF12C03E02FE130E04FEFE3
:1085E0005FEF6AEA70E080EF90E00E94DF058AEBBF
:1085F00092E0EED480939B060F91FF90EF90089548
:10860000EF92FF920F93E0909B06F12C03E02FE195
:1086100030E04FEF5FEF6AEA70E080EF90E00E9499
:10862000DF050F91FF90EF900895C098AB9AAF9A35
:108630008FB9779BFECF8FB1089587E087BBC09A33
:10864000AB9AAF9A83E58DB91EB880E8EEDF80E083
:10865000ECDF80E0EADF8AE18A95F1F700C0089557
:10866000EF92FF920F931F93CF93DF9300D000D030
:10867000CDB7DEB77C018B01A895AB9AAF9A1C826F
:108680001B821A82198280EDD0DF80E0CEDF8FB1AD
:1086900090E09C838B838B819C81982F88279C837F
:1086A0008B8380E0C2DF2FB18B819C81822B9C83E6
:1086B0008B838B819C8133E0969587953A95E1F782
:1086C0009C838B8387EC90E00197F1F700C000005A
:1086D00080E9ABDF80E0A9DF8FB190E09A838983E6
:1086E00089819A81982F88279A83898380E09DDFEA
:1086F0002FB189819A81822B9A83898389819A817A
:1087000053E0969587955A95E1F79A8389838B81F3
:108710009C81F7019183808389819A81F8019183FB
:1087200080830F900F900F900F90DF91CF911F914A
:108730000F91FF90EF90089570D088F09F5790F0C0
:10874000B92F9927B751A0F0D1F0660F771F881F76
:10875000991F1AF0BA95C9F712C0B13081F077D0DD
:10876000B1E0089574C0672F782F8827B85F39F07B
:10877000B93FCCF3869577956795B395D9F73EF4D5
:1087800090958095709561957F4F8F4F9F4F08957D
:10879000E89409C097FB3EF490958095709561959B
:1087A0007F4F8F4F9F4F9923A9F0F92F96E9BB2751
:1087B0009395F695879577956795B795F111F8CFCD
:1087C000FAF4BB0F11F460FF1BC06F5F7F4F8F4F38
:1087D0009F4F16C0882311F096E911C0772321F02E
:1087E0009EE8872F762F05C0662371F096E8862FC6
:1087F00070E060E02AF09A95660F771F881FDAF71D
:10880000880F9695879597F9089557FD9058440FCE
:10881000551F59F05F3F71F04795880F97FB991FDF
:1088200061F09F3F79F0879508951216130614069C
:10883000551FF2CF4695F1DF08C016161706180629
:10884000991FF1CF86957105610508940895E89404
:10885000BB2766277727CB0197F908950BD078C0FF
:1088600069D028F06ED018F0952309F05AC05FC087
:108870001124EECFCADFA0F3959FD1F3950F50E0FE
:10888000551F629FF001729FBB27F00DB11D639FC2
:10889000AA27F00DB11DAA1F649F6627B00DA11D68
:1088A000661F829F2227B00DA11D621F739FB00D0E
:1088B000A11D621F839FA00D611D221F749F33277E
:1088C000A00D611D231F849F600D211D822F762F17
:1088D0006A2F11249F5750408AF0E1F088234AF014
:1088E000EE0FFF1FBB1F661F771F881F9150504060
:1088F000A9F79E3F510570F014C0AACF5F3FECF37B
:10890000983EDCF3869577956795B795F795E7954B
:108910009F5FC1F7FE2B880F911D9695879597F95C
:10892000089597F99F6780E870E060E008959FEFF1
:1089300080EC089500240A941616170618060906F6
:10894000089500240A9412161306140605060895C5
:10895000092E0394000C11F4882352F0BB0F40F44D
:10896000BF2B11F460FF04C06F5F7F4F8F4F9F4F8D
:108970000895AA1BBB1B51E107C0AA1FBB1FA61766
:10898000B70710F0A61BB70B881F991F5A95A9F7B8
:1089900080959095BC01CD010895EE0FFF1F002436
:1089A000001C0BBE0790F691E02D0994A29FB00128
:1089B000B39FC001A39F700D811D1124911DB29F13
:1089C000700D811D1124911D0895BB274A3031F48B
:1089D000992322F4BDE2909581959F4F01C0BB275A
:1089E000FB015527AA27880F991FAA1FA41710F06B
:1089F000A41B83955051B9F7A05DAA3308F0A95D77
:108A0000A193009779F7B111B1931192CB0126C2CE
:108A1000CF93DF93CDB7DEB7AE014B5F5F4FFA0167
:108A200061917191AF0180919F069091A00603D052
:108A3000DF91CF9108952F923F924F925F926F9264
:108A40007F928F929F92AF92BF92CF92DF92EF92DE
:108A5000FF920F931F93CF93DF93CDB7DEB72B9782
:108A60000FB6F894DEBF0FBECDBF6C017B018A014B
:108A7000FC0117821682838181FFBFC1CE0101965E
:108A80003C01F6019381F70193FD859193FF81915C
:108A90007F01882309F4ADC1853239F493FD8591B6
:108AA00093FF81917F01853221F4B60190E0E6D1F8
:108AB000E8CF912C212C312CFFE1F315D8F08B322B
:108AC00079F038F4803279F08332A1F4232D2061DB
:108AD0001DC08D3261F0803369F4232D216016C0F2
:108AE000832D8260382EE32DE4603E2E2AC0F32DC4
:108AF000F8601DC037FC2DC020ED280F2A3040F053
:108B00008E32B9F436FC75C1232D2064322E19C083
:108B100036FE06C08AE0989E200D1124922E11C0C8
:108B2000EAE02E9E200D1124222EF32DF0623F2E1E
:108B300008C08C3621F4832D8068382E02C0883618
:108B400041F4F70193FD859193FF81917F0181119C
:108B5000B3CF982F9F7D9554933028F40C5F1F4F0F
:108B60009FE399830DC0833631F0833771F08335ED
:108B700009F055C020C0F801808189830E5F1F4F26
:108B800088248394912C530112C02801F2E04F0EE7
:108B9000511CF801A080B18036FE03C0692D70E041
:108BA00002C06FEF7FEFC5014ED14C018201F32D62
:108BB000FF773F2E15C0280122E0420E511CF8011C
:108BC000A080B18036FE03C0692D70E002C06FEF57
:108BD0007FEFC5012DD14C01F32DF0683F2E8201AE
:108BE00033FC19C0822D90E088169906A0F4B601D6
:108BF00080E290E043D12A94F5CFF50137FC8591CE
:108C000037FE81915F01B60190E038D121102A949E
:108C100021E0821A91088114910479F7E1C0843629
:108C200011F0893639F5F80137FE07C0608171818E
:108C3000828193810C5F1F4F08C060817181072E74
:108C4000000C880B990B0E5F1F4FF32DFF763F2E04
:108C500097FF09C090958095709561957F4F8F4FD4
:108C60009F4FF0683F2E2AE030E0A30143D1882EC9
:108C7000861844C0853731F4232D2F7EB22E2AE08A
:108C800030E025C0932D997FB92E8F36C1F018F4AE
:108C9000883579F0AEC0803719F0883721F0A9C047
:108CA000E92FE061BE2EB4FE0DC0FB2DF460BF2E97
:108CB00009C034FE0AC0292F2660B22E06C028E063
:108CC00030E005C020E130E002C020E132E0F801F0
:108CD000B7FE07C060817181828193810C5F1F4F55
:108CE00006C06081718180E090E00E5F1F4FA3019C
:108CF00001D1882E8618FB2DFF773F2E36FE0DC042
:108D0000232D2E7FA22E891458F434FE0BC032FC82
:108D100009C0832D8E7EA82E05C0B82CA32C03C0BD
:108D2000B82C01C0B92CA4FE0FC0FE01E80DF11D46
:108D30008081803321F49A2D997EA92E09C0A2FE4C
:108D400006C0B394B39404C08A2D867809F0B39416
:108D5000A3FC10C0A0FE06C0B21480F4280C922C14
:108D60009B180DC0B21458F4B60180E290E086D092
:108D7000B394F8CFB21418F42B1802C0982C212CFD
:108D8000A4FE0FC0B60180E390E078D0A2FE16C02A
:108D9000A1FC03C088E790E002C088E590E0B6013E
:108DA0000CC08A2D867851F0A1FE02C08BE201C072
:108DB00080E2A7FC8DE2B60190E060D0891430F427
:108DC000B60180E390E05AD09A94F8CF8A94F301E8
:108DD000E80DF11D8081B60190E050D08110F6CFF2
:108DE000222009F44ECEB60180E290E047D02A94CA
:108DF000F7CFF6018681978102C08FEF9FEF2B9608
:108E00000FB6F894DEBF0FBECDBFDF91CF911F919B
:108E10000F91FF90EF90DF90CF90BF90AF909F9019
:108E20008F907F906F905F904F903F902F9008951C
:108E3000FC010590615070400110D8F78095909525
:108E40008E0F9F1F0895FC0161507040019001102A
:108E5000D8F7809590958E0F9F1F0895DC01FC0137
:108E6000672F71917723E1F7329704C07C916D935E
:108E700070836291AE17BF07C8F308950F931F93D5
:108E8000CF93DF93FB01238121FD03C08FEF9FEF81
:108E90002CC022FF16C0468157812481358142179C
:108EA000530744F4A081B1819D012F5F3F4F31836F
:108EB00020838C93268137812F5F3F4F3783268312
:108EC00014C08B01EC01FB010084F185E02D0995B4
:108ED000892BE1F6D80116968D919C9117970196F2
:108EE00017969C938E931697CE01DF91CF911F9189
:108EF0000F910895FA01AA27283051F1203181F10C
:108F0000E8946F936E7F6E5F7F4F8F4F9F4FAF4F91
:108F1000B1E03ED0B4E03CD0670F781F891F9A1FA4
:108F2000A11D680F791F8A1F911DA11D6A0F711D58
:108F3000811D911DA11D20D009F468943F912AE064
:108F4000269F11243019305D3193DEF6CF0108954C
:108F5000462F4770405D4193B3E00FD0C9F7F6CF7D
:108F6000462F4F70405D4A3318F0495D31FD405245
:108F7000419302D0A9F7EACFB4E0A69597958795DB
:108F800077956795BA95C9F70097610571050895BA
:108F90009B01AC010A2E0694579547953795279566
:108FA000BA95C9F7620F731F841F951FA01D0895FE
:108FB000DC01CB01FC01E199FECF06C0FFBBEEBB9B
:108FC000E09A31960DB20D9241505040B8F7089595
:108FD000E199FECF9FBB8EBBE09A99278DB3089590
:108FE000A8E1B0E042E050E0E5CFDC01CB0102C0F7
:108FF0002D9105D041505040D8F70895262FE19982
:10900000FECF9FBB8EBB2DBB0FB6F894E29AE19AC0
:109010000FBE01960895F2DF272FF1CFF894FFCF0E
:109020000000000200000000DE07000000005754AE
:109030003D2025750A47530047533D2025750A53A7
:109040004E00534E3D2025750A454E4400574B3D7A
:109050002025750A565000503D332E360A520052D4
:109060004C3D2025750A68004F3D73740A53004734
:109070003D73740A530053523D53746174696F6EAB
:10908000200A57500057503D536E36332F506233ED
:10909000370A57540057503D536E41670A575400E2
:1090A00057503D50726F66696C65300A57540057CF
:1090B000503D50726F66696C65310A5754005750C5
:1090C0003D50726F66696C65320A57540057503DC7
:1090D00050726F66696C65330A57540057503D50A3
:1090E000726F66696C65340A57540057503D507270
:1090F0006F66696C65350A57540053523D55506888
:109100006561746572200A57500053523D50726574
:10911000686561746572200A57500053523D4D6175
:109120006E75616C200A57500053523D5265626F54
:109130006C6C696E67200A57500053523D43686952
:109140007068656174696E67200A57500053523D1C
:1091500050434268656174696E67200A5750005336
:10916000523D5043200A575000C2FBE1E5F0E8F2BF
:10917000E520E2FBF1EEF2F30056312E337A0020C7
:109180002020C2F0E5ECFF20F0E5E1EEEBEBE8EDAE
:10919000E3E02020202000C2FBE1E5F0E8F2E5203A
:1091A000F0E5E6E8EC00D2E5ECEFE5F0E0F2F3F014
:1091B000E020EFEEEBEEF7EAE8202000EDE8E7E054
:1091C00020EFF0E820E4EEEDE0E3F0E5E2E500D2A8
:1091D000E5ECEFE5F0E0F2F3F0E020F3E2E5EBE8B8
:1091E000F7E5EDE8FF00202020202020E4EEEDE070
:1091F000E3F0E5E2E020202020202000C4EBE8F2AC
:10920000E5EBFCEDEEF1F2FC20E2EFE8F2FBE2E050
:10921000EDE8FF00D4F3EDEAF6E8FF20E4EEEDEE32
:10922000E3F0E5E2E000EDE8E6EDE5E3EE20EDE079
:10923000E3F0E5E2E0F2E5EBFF2020202000CCE0C7
:10924000EAF1E8ECE0EBFCEDE0FF20ECEEF9EDEE0E
:10925000F1F2FC202000E2E5F0F5EDE5E3EE20ED93
:10926000E0E3F0E5E2E0F2E5EBFF20202000CCE0D7
:10927000EAF1E8ECE0EBFCEDE0FF20ECEEF9EDEEDE
:10928000F1F2FC202000E2E5F0F5EDE5E3EE20ED63
:10929000E0E3F0E5E2E0F2E5EBFF20202000D2E59C
:1092A000ECEFE5F0E0F2F3F0E020E2EAEBFEF7E5C8
:1092B000EDE8FF202000CAEEEDF2F0EEEBFC20EF2F
:1092C000EE20E2E5F0F5F320202020202000EDE85C
:1092D000E6EDE5E3EE20EDE0E3F0E5E2E0F2E5EBDC
:1092E000FF2020202000CAEEFDF4F4E8F6E8E5EDCA
:1092F000F220EFF0EEF4E8EBFF2020202000E2E582
:10930000F0F5EDE5E3EE20EDE0E3F0E5E2E0F2E597
:10931000EBFF20202000CAEEFDF4F4E8F6E8E5EDCE
:10932000F220EFF0EEF4E8EBFF2020202000EDE04B
:10933000E3F0E5E2E0F2E5EBFF202000D2E5ECEF20
:10934000E5F0E0F2F3F0E020EDE8E6EDE5E3EE2015
:1093500020202000EFE0E9EAE82000D2E5ECEFE58C
:10936000F0E0F2F3F0E020ECE5F1F2E02020202044
:109370002000C2FBE1E5F0E8F2E520EFF0EEF4E8D2
:10938000EBFC00CFF0EEF4E8EBFC203500CFF0EE84
:10939000F4E8EBFC203400CFF0EEF4E8EBFC2033F3
:1093A00000CFF0EEF4E8EBFC203200CFF0EEF4E872
:1093B000EBFC203100CFF0EEF4E8EBFC2030005362
:1093C0006E416700536E506200CAEEECEFFCFEF295
:1093D000E5F000C4EEEF2E20EDE0F1F2F0EEE9EA68
:1093E000E800EFEBE0F20020D1F3F8EAE020EFEB49
:1093F000E0F22000ECE8EAF0EEF1F5E5EC00D1F364
:10940000F8EAE000D0E5E1EEEBEBE8EDE32000D098
:10941000F3F7EDEEE9002020D0F3F7EDEEE92020A0
:109420002000CDE8E6EDE8E920EDE0E3F02E2000B5
:10943000C2E5F0F5EDE8E920EDE0E3F02E002020B4
:10944000D1F2E0EDF6E8FF00E2E5F0F5E000EDE84E
:10945000E7E000CCEEF9EDEEF1F2FC00CFF0E8ED44
:10946000FFF2EE202000C2DBC1D0C0D2DC00C2DBA4
:10947000CACB00C2CACB00CDE0F1F2F0EEE8F2FCBC
:1094800000C7E2F3EAEEE2FBE520F1E8E3EDE0EB12
:10949000FB00CFF0E5E4F3F1F2E0EDEEE2EAE80004
:1094A000D3ECEEEBF7E0EDE8FF00C2F0E5ECFF20D7
:1094B000EFE0E9EAE80020C4E0F2F7E8EA20EDE8AE
:1094C000E62E20EDE0E3F0E5E2E0F2E5EBFF002040
:1094D000C4E0F2F7E8EA20ECE5F1F2E020EFE0E9A1
:1094E000EAE800F0F3F7EDEEE900EDE8E6EDE8E993
:1094F00000EDE0E3F02E00C2E5F0F5EDE8E900C292
:06950000DBD5CEC4000023
:00000001FF
